:100000006EC40000A4C40000A2C40000A0C400008C
:100010009EC400009CC400009AC4000098C4000064
:1000200096C4000094C400000C9471300C945931B3
:100030000C9426308CC400008AC4000088C40000E0
:1000400086C4000084C4000082C4000080C4000094
:100050007EC400000C944D307AC4000078C40000C7
:1000600076C4000074C4000072C4000070C40000B4
:100070006EC400006CC400006AC4000068C40000C4
:1000800066C4000064C4000062C4000060C40000D4
:100090005EC400005CC400005AC4000058C40000E4
:1000A00056C4000054C4000052C400000501098079
:1000B000A101850319012AB700150126B700950192
:1000C00075108100C0050C0901A101850419012AE0
:1000D000A002150126A002950175108100C005013E
:1000E0000906A1018506050719E029E71500250184
:1000F0009508750181020507190029EF15002501F2
:1001000095F075018102050819012905950575010C
:100110009102950175039101C00660FF0961A1017B
:100120000962150026FF00952075088102096315F4
:100130000026FF00952075089102C005010906A15F
:1001400001050719E029E7150025019508750181CA
:10015000029501750881010507190029FF15002680
:10016000FF0095067508810005081901290515008D
:100170002501950575019102950175039101C00056
:10018000000000000000000000000000000000006F
:10019000000000000000000000000000000000005F
:1001A0000000007E0F00D4FFFFFFC70000007800B2
:1001B000000000000000002A2B28000000000000C2
:1001C0000000000000000000000029000000002CDA
:1001D0001E3420212224342627252E362D37382779
:1001E0001E1F202122232425263333362E37381F85
:1001F0000405060708090A0B0C0D0E0F1011121347
:100200001415161718191A1B1C1D2F3130232D35E4
:100210000405060708090A0B0C0D0E0F1011121326
:100220001415161718191A1B1C1D2F3130354C09BF
:10023000025B00030100A0FA0904000001030101B0
:100240000009211101000122440007058103080073
:10025000010904010002030000000921110100014D
:100260002222000705820320000107050303200066
:10027000010904020001030000000921110100012D
:10028000226D000705840320000112010002000016
:100290000008167500700100010203011C037600BE
:1002A000690061006C003A006600360034006300AB
:1002B00032006200330063000000160342006C004D
:1002C000610063006B002000450036002E00350001
:1002D0000000180348006F00720072006F00720087
:1002E000540072006F006C006C00000004030904ED
:1002F00029001E001F0020002100220023002400EE
:100300002500260027002D002E0035002A002B0096
:1003100014001A000800150017001C0018000C003B
:10032000120013002F00300028004B003900040099
:100330001600070009000A000B000D000E000F0058
:1003400033003400310000004E00E100E1001D00E8
:100350001B000600190005001100100036003700D0
:100360003800E50052002152E000E300E200000006
:10037000000000002C000000E6002152E4005000C4
:1003800051004F004C00007C3A003B003C003D0017
:100390003E003F0040004100420043004400450051
:1003A00001000100207821782378247825782678A8
:1003B00027782878010001000100010001000100F8
:1003C0004A00027802780378047805780100010079
:1003D00001000100010001000100010000004D00CA
:1003E0000100010001000100010001000100010005
:1003F00001000100010001000100010001000100F5
:1004000001000100000000000000010000000100E8
:100410000100010001000100010046002223252601
:1004200028292A2C2D2F3032333536383A3B3D3EA1
:100430004042434547494A4C4E5051535557595AEB
:100440005C5E6062646668696B6D6F717375777905
:100450007B7D7F81838587898A8C8E909294969804
:100460009A9C9E9FA1A3A5A7A8AAACAEAFB1B3B416
:10047000B6B8B9BBBCBEBFC1C2C3C5C6C7C9CACB6B
:10048000CCCDCED0D1D2D2D3D4D5D6D7D7D8D9D936
:10049000DADADBDBDBDCDCDCDCDCDDDDDDDDDCDC9F
:1004A000DCDCDCDBDBDBDADAD9D9D8D7D7D6D5D4BC
:1004B000D3D2D2D1D0CECDCCCBCAC9C7C6C5C3C288
:1004C000C1BFBEBCBBB9B8B6B4B3B1AFAEACAAA8DD
:1004D000A7A5A3A19F9E9C9A98969492908E8C8A91
:1004E00089878583817F7D7B79777573716F6D6B6C
:1004F0006968666462605E5C5A5957555351504E44
:100500004C4A4947454342403E3D3B3A38363533F5
:1005100032302F2D2C2A292826252322FFAA7F5569
:100520004000010101010101010101020202020278
:10053000020202020303030303030303040404048B
:100540000404040505050505060606060607070753
:10055000070708080808090909090A0A0A0B0B0B0A
:100560000C0C0C0D0D0D0E0E0E0F0F0F10101111A7
:10057000111212131314141515161617171818192B
:10058000191A1A1B1B1C1D1D1E1E1F202021222292
:10059000232424252626272829292A2B2C2D2D2ED5
:1005A0002F30313232333435363738393A3B3C3DEF
:1005B0003E3F404142434445464748494A4C4D4EE0
:1005C0004F50515354555658595A5B5D5E5F6162A6
:1005D00064656668696B6C6D6F7072737577787A35
:1005E0007B7D7E8082838587888A8C8E8F91939590
:1005F00096989A9C9EA0A2A3A5A7A9ABADAFB1B3B4
:10060000B5B7BABCBEC0C2C4C6C9CBCDCFD1D4D693
:10061000D8DBDDDFE2E4E7E9EBEEF0F3F5F8FAFD35
:10062000FF1E0F0500047F3F1F64321464321478EC
:100630003C1E1E140A05FD377A585A000004E6D6FF
:10064000B4460200210116000000742FE5A3E00863
:100650004A023F5D003D8889C65436C3174FE4DD2A
:10066000E515CFD3198E5891B26DBD6AB0C0EBFAC3
:10067000BA054041350FA89BC160D4FC50A8C8FF03
:100680009275AD101EE45224B2FA85420D391F61F5
:10069000060BE30903E2A90B59A1FD96ACE63A6902
:1006A0009AD7ACF90FD4EF8E44835A7D1C6D935CBE
:1006B00023B8AB0E09238493286D058A643BC828B0
:1006C00047BA9FABFE723196A263653B4C425C1900
:1006D00062529C3F3C5BFCB01482B2F7313CA4A355
:1006E000C93412B442C155A1546459691E7F0343F1
:1006F00014FB119D5B971FAAA1A741558CEAA1107D
:10070000FD1C825CB15ED61B63956F349793F3F248
:100710002B69D1BC7B65ACF5FE463A1ACC6A5826EB
:100720009B5444FFADB2DFE7792F1EE0244C2F012C
:100730000C79B30E7231D69F0CC9E9B8C7CA062D21
:10074000093CBE55276707FB30EF6F02714A3CBE7C
:10075000DFF2FBCC886F09939CEB267B0BCCDB7222
:10076000AF2A77B316C04BEB66FB4218B80C176E76
:10077000A3CF53469293A2C9F327CD585A8CC4D223
:10078000F727E683E5324C0331EF81ECF9A89CE2D0
:10079000F0218C1569067EB4784D2CF957A8870690
:1007A0006E4570420DD0E53C1EB012552AFC385BF8
:1007B00057E89EBB6280942C135D39C0524BF933CD
:1007C00073D1D0FBF5D09EE7F4A1FFD7B289C3E87F
:1007D00031EC893CEF46E73AB7D1A48D934E2FEF29
:1007E000C761EB78D4DFC878FEE55D50823F118C9D
:1007F000C41E7D730B6E1BF0DFA1FF42E553749E98
:1008000092C61F171E6664B0D038380B8DB906111A
:10081000A72721F8ABC68A4BB522850309FD3D6C9D
:10082000F7CA819F3D340DB17F124C34A8D7C26105
:1008300078767367AAA8D6F225C858DF7C75D9FAEE
:10084000A3E107CC89AFAC43473EFFA58D81DE3BDA
:10085000B6D89B20F0005E8D03DAB4F9748DC343E3
:10086000CFF841C2BB6580E90F4C5A60F9952C3F27
:1008700088F6F2704D55B7D24D3112F91984E5184A
:10088000F7B634182D4022DCFEE4B8C2532FFBB576
:10089000D60D08000000D48E19CA1717F37A00018C
:1008A000DB04CB100000865446F3B1C467FB0200A2
:1008B00000000004595A504F52514A4D4B4E2A4C99
:1008C0002F30B6B7ABACBBBCA9AABDBE0D0E0B0F8B
:1008D0001A0508050905071811130408120C11243C
:1008E0001FBECFEFDAE0DEBFCDBF04B603FE18C0F7
:1008F0008091420590914305A0914405B091450532
:100900008730904BA740B04B59F41092420510929B
:1009100043051092440510924505E0E0F8E309957F
:1009200025E0A6EEB1E001C01D92A234B207E1F7C6
:1009300011E0A0E0B1E0E8E5F8E602C005900D9214
:10094000A63EB107D9F70E940C290C94CB3358CBA3
:100950009C01FB019A9581159F4120F5832F8170A1
:10096000B32FB270AA27732F74706627532F587055
:10097000442734FF0DC08295807FAB2B09F0806245
:10098000672B09F08064452B09F08068099508956C
:10099000AB2B09F08260672B09F08460452BB1F323
:1009A0008860F4CF80E0F2CF0C94F9310895982F4D
:1009B00092959F7024E0911102C020E0982F892F1A
:1009C00086958695811511F02E5F982F892F869533
:1009D000820F089581FF02C0479A089547980895AD
:1009E00080933E05089580933F05089521E030E00F
:1009F00001C0220F8A95EAF780913F05822BF3CF41
:100A000021E030E0A90102C0440F551F8A95E2F7AA
:100A1000CA01809590913F058923E5CF292F953014
:100A200090F58F3080F590E03FE0239F800D911D81
:100A30001124282F277041E001C0440F2A95EAF7BE
:100A400023E0969587952A95E1F7FC01EE0FFF1FAD
:100A5000E80FF91FEA50FC4F20E030E070E05191C0
:100A6000DF01CB01022E02C0969587950A94E2F72A
:100A7000817081958527842385278E932F5F3F4F33
:100A80002330310561F70895292F953078F58F309F
:100A900068F590E03FE0239F800D911D1124682FA1
:100AA000677023E0969587952A95E1F7FC01EE0F94
:100AB000FF1FE80FF91FEA50FC4F40E050E080E0D4
:100AC000219130E0062E02C0369527950A94E2F770
:100AD00021703327042E01C0220F0A94EAF7822BDB
:100AE0004F5F5F4F4330510559F7089580E00895F7
:100AF00090913F0521E030E0F90101C0EE0F8A95A9
:100B0000EAF7D90102C0AA0FBB1F6A95E2F7EA2BE8
:100B100001C0220F4A95EAF7892F8E23E81303C0FC
:100B2000892F822B60CF2095822F8923FBCF809144
:100B3000A4039091A303981301C008958F5F877059
:100B4000FACF90918A048095892380938A04282F74
:100B50002770211110C0891771F09091410592FF03
:100B60000AC08695869586954BDF10928A0410926E
:100B70008C0410928B040895982F9095809187048F
:100B8000892380938704089580918604811531F02C
:100B90001092860410928E0410928D040895803E67
:100BA0009105D9F1C8F48133910509F482C048F464
:100BB0008932910509F472C08A32910509F480C026
:100BC000089589339105E9F082389105D1F0853394
:100BD000910509F45EC00895843E9105D9F148F469
:100BE000823E910539F1833E910549F181EE90E015
:100BF0000895863E9105C9F1873E910509F43EC0EE
:100C00000895209140052370211164C02091410571
:100C100023FF14C089E290E008952091400520FD53
:100C200045C03091410530FF09C024FD24C083EE4A
:100C300090E008952091400522FDF7CF089520917E
:100C4000400522FD44C03091410530FD43C024FFE2
:100C5000F5CF11C02091410521FFF0CF80914005D3
:100C600084FD09C087EE90E008952091400523FFA0
:100C7000E5CF24FFF7CF80E090E008952091400574
:100C800023FD2BC03091410531FFE1CF84EE90E090
:100C900008952091400525FFD1CFBCCF209140057C
:100CA00025FD1EC02091410523FFC8CF89E390E0B8
:100CB00008952091400526FFC1CF8AE290E0089573
:100CC0002091400526FFBACF81E390E0089582EE9F
:100CD00090E0089580EE90E0089586EE90E008950B
:100CE00085E390E008959091400592FF10C041E0A7
:100CF000282F2471243009F040E031E0282F28719A
:100D0000283009F030E0431711F02CE0822793FFE0
:100D100010C041E0282F2471243109F040E031E077
:100D2000282F2871283109F030E0431711F02CE00A
:100D300082273091410530FF10C051E0282F2171EA
:100D4000213009F050E041E0282F2871283009F0C7
:100D500040E0541711F029E0822731FF10C041E034
:100D6000282F2171213109F040E031E0282F28712E
:100D7000283109F030E0431711F029E0822794FD73
:100D8000877E08951F93CF93DF9309DFEC018115D0
:100D900022E5920708F052C0811540E5940708F05B
:100DA000CDC0803E910520F58D3C910508F0A1C095
:100DB000883A910570F4853A910508F097C0813022
:100DC0009105B9F10497813A910598F1C0E0D0E01E
:100DD00030C0885A91094B97C8F7C85AD0E0CC0F59
:100DE000DD1FC658DE4F0990D881C02DD46421C0C4
:100DF000811550E49507B0F4C11580E2D80708F0DA
:100E0000B3C0C83ED105A8F0CE019A9581159F4187
:100E1000E8F68D2F68DF182FCE019927C0DEEC0190
:100E2000D12B07C09927BBDECC27DF70C82BD92B6D
:100E3000D06ACE01DF91CF911F910895803842E5AD
:100E40009407C8F5803652E5950708F05BC0C034BA
:100E500082E5D807D0F4C03292E5D90708F04BC03C
:100E60008C2F8695869520E2829FC0011124C37045
:100E700021E030E0A90102C0440F551FCA95E2F7F6
:100E8000EA01C82BD92BDD68D4CF8C2F86958695A7
:100E9000877050E2859FC0011124C37021E030E0CB
:100EA000A90102C0440F551FCA95E2F7EA01C82BF9
:100EB000D92BDC68BECF803C52E5950758F48F7182
:100EC000C03AD245A0F590E0982F8827EC01C46F76
:100ED000D06AAFCF805C9245809708F077CFDC2F47
:100EE000CC27CC27DF71C06FD06AA3CFA497D06482
:100EF000A0CFD0659ECFCF71D0E0DC2FCC27C16FC3
:100F0000D06A97CF86958695877020E2829FC00130
:100F10001124C37021E030E0A90102C0440F551F25
:100F2000CA95E2F7EA01C82BD92BDA6882CFDBDE5B
:100F3000C82FD0E0DC2FCC27D0627BCF8F71D3DEDF
:100F400093E0CC0FDD1F9A95E1F7CC27DF70282FB7
:100F500030E084FF05C050E1859F900111243327C4
:100F6000C22BD32BD06965CF8D2F8F71BCDE182F8C
:100F7000CE01992714DEEC01D12BDECF80E008955D
:100F8000F894E82FE295EF70F0E041A18F7021E036
:100F900030E0B90102C0660F771F8A95E2F7CB01F6
:100FA000962F9095942391A392A1892B82A3789454
:100FB00008950895CF92DF92EF92FF921F93CF93FF
:100FC000DF93172FE82FF0E0EF5DFA4F71110CC09F
:100FD000E4918E2F7E2F6E2FDF91CF911F91FF9086
:100FE000EF90DF90CF900895E62EF12CC72ED12CF4
:100FF000F491EF2F86E0689F90011124CFEFD0E0AD
:10100000C901BE010E94CC31AB01EE0CFF1C65E5AD
:10101000649FC001659F900D1124E81AF90A6E2D96
:10102000660F6E0D7E01EC18FD08FE9DD001FF9D40
:10103000B00D11248B2F169F70011124EF2CFF246B
:101040006E01CE18DF087601FE9D6001FF9DD00C79
:1010500011247E01E61AF108B701169F7001179F4F
:10106000F00C1124EF2CFF24CE19DF09FC9F700136
:10107000FD9FF00C11247F2D43305105C1F02C3F12
:10108000334058F441305105B1F04230510509F078
:10109000A2CFEB2F8F2D7F2F9ECF4430510571F0C3
:1010A0004630510509F497CF7B2F8D2D94CF7D2DA0
:1010B000EB2F8F2F90CF7F2FED2D8DCFEF2D7B2F0F
:1010C000F8CFCF93982F762F842FC22F692F72DFFE
:1010D000472F282F8C2F90E0E9D2CF91089580914F
:1010E0007D04843028F48370846080937D040895A7
:1010F0008C3AE8F38370886AF8CFCF93DF938091BE
:101100007D0480FD0BC0C0E0D0E020E040E060E066
:10111000CE01CCD22196C831D105B9F719D6DF91CD
:10112000CF910895FF920F931F93CF93DF93182FC2
:10113000062FF42E80917D0480FF0CC0C0E0D0E02B
:101140002F2D402F612FCE01B1D22196C831D1056C
:10115000B9F7D3DFCDB7DEB7E5E00C944532CF93D6
:10116000DF93EC01209180049C81892F817090FD98
:10117000822F692F627091FD622F492F447092FD7A
:10118000422FD0DF8C8190E00196877099278C8365
:10119000DF91CF910895982F762F842F20917D0491
:1011A00020FF07C0692F06DF962F672F482F892F52
:1011B000B9CF0895CF93DF93EC01EDE7F4E04381DD
:1011C00062818C81E8DF8C818F5F8C83DF91CF918E
:1011D0000895CF93DF93EC01EC81F0E0E45EFB4FE8
:1011E0004491EDE7F4E062818181D5DF8C818F5FEE
:1011F0008C83DF91CF910895FF920F931F93CF932C
:10120000DF93EC01F12C00E010E08C81980140911B
:10121000800460917F048F0D54DF0F5F1F4F8AE0C1
:10122000F80E0831110589F768DF8C819A8190FFEB
:1012300007C08F5F8C83CDB7DEB7E5E00C944532F5
:101240008150F8CFEF92FF920F931F93CF93DF93CC
:10125000FC018281FF24F39480FF02C0FF24FA94F2
:10126000C0E0D0E020E040E060E0CE011FD204E02A
:1012700010E0E12C809142038E0D89318CF168E100
:101280000E94BF31892F082E001C00088C170D0604
:1012900079F4409180040403A001112455954795E9
:1012A000559547959E0160917F0480917E0409DFEA
:1012B000EF0C01501040F1F62196C831D10591F69E
:1012C0001CDF80914203F1E0FF120EC0811591F006
:1012D000815080934203CDB7DEB7E6E00C944432F0
:1012E00087FFD1CF885ECFCF90E00196BE010E94EC
:1012F000E031EFCF87E1EDCFCF93DF93C0E0D0E0D7
:1013000020E040E060E0CE01D1D12196C831D10586
:10131000B9F7C0E0D0E080914103082E001C00081E
:10132000C817D0055CF180910601082E001C00084A
:101330008C170D061CF19E014091800460917F0482
:1013400080917E04BEDE2196C831D10521F7D5DE1D
:101350008091050190914103980F90934103209152
:101360000601280F20930601121614F497311CF081
:10137000819580930501DF91CF91089520E040E0B1
:1013800060E0CE0193D1DFCFA6E0B0E0EAECF9E077
:101390000C9426328D839E83AD81BE811496FC9180
:1013A0002F2F30E0D9010E94BC339B01AC010E9479
:1013B0008A336B017C0180E290E09C012F1B310994
:1013C000F901A5E5B0E0A70196010E948A3369837F
:1013D0007A838B839C839F01DF010E9410329B01E3
:1013E0000E9416329B01AC012C0D3D1D4E1D5F1D50
:1013F00069817A818B819C810E949A33022F30E02F
:101400000A32A0F5A901440F551F420F531F5595ED
:101410004795142F1095E12CF12C85E5D82ED01A84
:101420008D2DE1FC802F9701412F60917F0449DED3
:101430003FEFE31AF30A88E1E816F10489F75DDE6D
:10144000AD81BE8114969C9181E0911519F0903286
:1014500019F48FEF8093040180910401890FED81CD
:10146000FE8184832696E8E00C94423285E590E084
:10147000821B930BAC01440F551F480F591F57FF98
:10148000C6CF4F5F5F4FC3CF0F931F93CF93DF93B1
:10149000EC0120E030E060917F0480917E049C812B
:1014A00089010F5F1F4F2C3031053CF4911541F03D
:1014B0004091800406DE9801EECF409180049111A6
:1014C00040E0FFDD98010831110529F716DE8C8117
:1014D00090E00196817099278C83DF91CF911F91C5
:1014E0000F910895A0E0B0E0E8E7FAE00C9426320E
:1014F000873080F581112FC0909180009F7D90935F
:1015000080002091860030918700A82FB0E00E94D3
:10151000BC3326E030E040E050E00E949A3369019D
:101520007A0180918600909187006CE070E00E94C3
:10153000CC316217730798F0C90169E070E00E942E
:10154000CC3170938B0060938A00CDB7DEB7E8E0B2
:101550000C94423286E0909180009062D0CF8091CE
:10156000860090918700009186001091870020915D
:10157000860030918700C6E0D0E0BE010E94CC31E9
:10158000C60ED71EE11CF11C85E0CC0CDD1CEE1C48
:10159000FF1C8A95D1F7C801BE010E94CC3140E002
:1015A00050E0260F371F411D511DC701B6010E9493
:1015B0009A3369017A01E0918600F0918700CA01AF
:1015C000B9010E94A4319B01AC01DF010E948A3362
:1015D0009B01AC01C701B6010E94A4312FE0969592
:1015E0008795779567952A95D1F720918600309158
:1015F0008700261737071806190608F0A2CF609152
:101600008600709187009DCF982F990F990F990FA1
:10161000209174042770922B9093740421E09830E9
:1016200008F420E09091740420FB90F990937404E6
:1016300059CFFB01811520E2920728F4811541E082
:10164000940738F408959C0130522115304348F036
:101650000895392F94FF02C03295307F2081232BCB
:10166000208399270895462B22FF0FC0982F92952B
:101670009F708F70892B962F92959F706F70692B3A
:10168000942F92959F704F70492B982F9623961305
:1016900009C050E04095509590E04823592381E0DF
:1016A000452B09F080E008956A9A0895FC01EE0F39
:1016B000FF1FE80FF91FEF5CFD4F6183408322831A
:1016C00008951092D0041092CF04EFE8F4E08581E1
:1016D000811102C014821682379684E0E73CF80735
:1016E000B1F70895AC013091D2046091D104232F59
:1016F000621301C00895822F90E0FC01EE0FFF1FDE
:10170000E953FB4F0190F081E02DE417F50791F4C8
:1017100067E0649FF001659FF00D1124E157FB4FD6
:1017200041E044832313E6CF019683709927809389
:10173000D20408950196282F2370DACF0F931F93B8
:10174000CF9301E010E0082E01C0000F0A94EAF7E1
:10175000C09185049C2F9023911115C090918A040B
:10176000969596959695891306C010928A041092C4
:101770008C0410928B043AD9C027C0938504CF9172
:101780001F910F9108953CD9F7CF90916904890278
:101790009001112437FF03C08093690408952F3707
:1017A00031051CF4980F9093690408959C0180E022
:1017B00090E0F901E80FF91FE491E41307C091E00C
:1017C0008927F901E80FF11D849108950196861784
:1017D00080F380E00895E0919903F0919A033097A7
:1017E00039F00190F081E02D309711F009950895BE
:1017F00080E00895A3E0B0E0E0E0FCE00C942C323F
:101800009C0180912E0290912F0282179307B1F0D4
:1018100030932F0220932E02E0919903F0919A03C6
:10182000309761F00084F185E02D309739F083E046
:1018300089833B832A83CE01019609952396E2E0B2
:101840000C944832A3E0B0E0E8E2FCE00C942C32C7
:101850009C0180912C0290912D0282179307B1F088
:1018600030932D0220932C02E0919903F0919A037A
:10187000309761F00084F185E02D309739F084E0F5
:1018800089833B832A83CE01019609952396E2E062
:101890000C94483290912001913091F0AAEEB1E081
:1018A000EFEF90E02D91821751F0EF3F19F42111E5
:1018B00001C0E92F9F5F9630A9F7EF3FC9F4089563
:1018C0009091400597FFEACFE82FE695E695E695DB
:1018D000803FA8F7F0E0E051FE4F877021E030E054
:1018E00001C0220F8A95EAF78281822B82830895B4
:1018F0000E2E000CFF0BE851FE4FF8CF9091200107
:10190000913021F49091400597FD0CC0EAEEF1E092
:101910009191891302C0DF011E9251E0E03FF5076B
:10192000B9F70895E82FE695E695E695803FC8F764
:10193000F0E0E051FE4F877021E030E0A90102C0E5
:10194000440F551F8A95E2F7CA0180959281892339
:101950008283089580911F0108952FB7F894809194
:10196000280290912902A0912A02B0912B022FBF48
:101970000895CF93DF93C091870480918904C82B89
:10198000809186048115F1F0E8DF20918D0430917B
:101990008E04821B930B8838934108F0F5D8D091C0
:1019A000860480912001813021F48091400587FDDB
:1019B0000DC086E02AEE31E090E0815058F491119C
:1019C000E3D8CD2B8C2FDF91CF9108958EE122EFBC
:1019D00031E0F2CFF90141919F01411571F39F5F11
:1019E000ECCF962F2091410522FF0FC0682F660F84
:1019F000660F660F692B60938A040E94F604ADDFC0
:101A000090938C0480938B0408950C94F604909129
:101A10008604292F2823211559F080958923809346
:101A20008604811531F099DF80938D0490938E04A4
:101A3000089580E090E0F8CF2FB7F89460912802E5
:101A40007091290280912A0290912B022FBF089554
:101A50000895FC019B0180911E0290911F02861740
:101A6000970740F0672B29F48091E8008E778093E8
:101A7000E800C90140E0009741F4411106C080919F
:101A8000E80082FF2FC080E00895209172032115A5
:101A9000A9F12530A9F12091E80023FD2DC0209166
:101AA000E80022FDECCF2091E80020FFE4CF309148
:101AB000F3002091F200009719F02830310558F01A
:101AC00041E02830310509F040E02091E8002E7710
:101AD0002093E800D0CF41914093F10001972F5F10
:101AE0003F4FE9CF80917203811541F0853041F07D
:101AF0008091E80083FFC3CF81E0089582E00895DC
:101B000083E008958091180287FF13C08091E80058
:101B100082FF06C08091E8008B778093E8000895EB
:101B2000809172038111F2CF089580917203811523
:101B3000D9F38091E80080FFF8CF8091E8008E779C
:101B4000ECCF2091E4003091E50095E6A9012091C9
:101B5000EC00822F817020FF06C08091E80080FF9A
:101B600006C080E008952091E80022FD1AC080910F
:101B70007203811589F0853089F08091EB0085FD35
:101B80000FC02091E4003091E50042175307F9F2AD
:101B90009A95E1F684E0089582E0089583E008953F
:101BA00081E00895E8EDF0E080818E7F80831092DF
:101BB000E2001092DA001092E100A0EEB0E08C9109
:101BC00081608C9380818F77808319BCA7EDB0E012
:101BD0008C918E7F8C9380818F7E808310921702F0
:101BE0000895E0919903F0919A03309739F00284B7
:101BF000F385E02D309711F060E209950895982F54
:101C00009093E900891771F07091EC002091ED003C
:101C10005091F00021FD09C09F5F973089F78093B4
:101C2000E9000895762F242F50E03091EB003E7F9D
:101C30003093EB003091ED003D7F3093ED0030911B
:101C4000EB0031603093EB007093EC002093ED00DB
:101C50005093F0002091EE0027FDDECF0895A0E024
:101C6000B0E0E5E3FEE00C942632C8EDD0E08881D8
:101C70008F7E8883E7EDF0E080818160808384E05F
:101C800082BF81E08093170288818E7F888302EE75
:101C900010E0F80110821092DA0081EEC82ED12CEB
:101CA000F601108288818F77888388818068888395
:101CB00088818F7D888319BC10927203109216025E
:101CC00010924F031092150290EEE92EF12CF701BD
:101CD00080818B7F808388818160888342E060E09F
:101CE00080E08DDFF60180818E7F8083F801808126
:101CF00081608083808188608083F70180818E7F0E
:101D00008083888180618883CDB7DEB7E8E00C945A
:101D10004232E091A4039091A30329E0E91302C0A9
:101D200080E00895AE2FB0E02E9FF0011124EB5516
:101D3000FC4F3181361306C03081381303C0358122
:101D4000341304C0FD013196E770E8CF81E00895B7
:101D50003EB13B7F2EB124604FB7F89481E392E00F
:101D6000FC010196508168E02EB9000000C057FFC9
:101D70003EB9550F000000C000C000C03EB900C011
:101D80006A9591F752E08937950751F74FBF8FE574
:101D900094E00197F1F700C00000089581E080937E
:101DA000E00080E28093D8001092C9008FE19EE4A9
:101DB0000197F1F700C0000087E090EBDC01809311
:101DC000420590934305A0934405B093450588E1EF
:101DD0009CE00FB6F894A895809360000FBE909396
:101DE0006000FFCF0F931F93CF93DF938B01EA0126
:101DF00090917203943051F58093E9008FEF9091A8
:101E0000E80095FD06C095ED9A95F1F700008A95DA
:101E1000B1F78091E80085FF19C093DE811111C0F0
:101E20008091E80085FD06C08091E8008E77809360
:101E3000E800F3CFF80181918F018093F1002197A1
:101E400079F78091E8008E778093E800DF91CF9159
:101E50001F910F910895792F603229F440E250E0EC
:101E6000682F82E0BFCF0895CF93DF93D82FC92F7B
:101E700048E050E0682F792F81E0B4DF88E0ED2F53
:101E8000FC2FA0E2B2E001900D928A95E1F7DF917C
:101E9000CF910895BC0140E250E084E0A3CFBC01A3
:101EA00043E050E084E09ECF9091410592FB2227D1
:101EB00020F9281779F080FB92F990934105609101
:101EC00040057091410584E090E00E94533382E028
:101ED0000C94A1050895FC01608186E090E00C94CB
:101EE00039331F93CF93DF93962F122F632F8430B4
:101EF000D8F49530C8F44F30B8F4C42FD0E0CC0FEC
:101F0000DD1F2EE1929FC00DD11D112496E9899FFE
:101F1000C00DD11D1124CE0189960E943933612F45
:101F2000CE018A960E943933DF91CF911F91089597
:101F300080912001813061F58091400587FF28C0A4
:101F400018DD8093F10140E250E069E773E080EF33
:101F500091E00E94F432892BD1F080E2E0EFF1E0D1
:101F6000A9E7B3E001900D928A95E1F7E09199031A
:101F7000F0919A03309759F00480F581E02D309765
:101F800031F086E08093F00180EF91E009950895AB
:101F9000F0DC8093E80148E050E06BE973E088EE04
:101FA00091E00E94F432892B91F388E0E8EEF1E0B1
:101FB000ABE9B3E001900D928A95E1F7E0919903C6
:101FC000F0919A03309719F30280F381E02D309756
:101FD000F1F288EE91E0DACFCF93C82F8115C1F0EE
:101FE0008CEF8C0F813A80F580912001813021F4B3
:101FF0008091400587FD0EC0EAEEF1E08191C8179F
:10200000F9F021E0E03FF207C9F78C2F43DC90DFC5
:10201000CF910895EC2FE695E695E695F0E0E05136
:10202000FE4F828190E04C2F477021E030E002C0EB
:10203000220F331F4A95E2F782239323892B29F33A
:102040008C2F5CDC75DFE1CF80E28C0F883068F488
:10205000C77081E090E001C0880FCA95EAF7C0918F
:102060008704C82BC0938704D2CF8BE58C0F8330B5
:1020700030F42C2F2452330BC901BCDBC9CFC85A12
:10208000CB3130F6EC2FF0E0EE0FFF1FE055FE4FA6
:1020900080819181D7DBBCCF811509F19CEF980F2E
:1020A000913A10F42BDC44CF90E2980F983050F422
:1020B000877091E001C0990F8A95EAF7892F0E94F5
:1020C000BC05F1CF9BE5980F933018F480E090E0C9
:1020D00091CB885A8B3118F480E090E0B3CB08950F
:1020E0001F93CF93DF93182FEB0176DF209731F406
:1020F000812FD2DFDF91CF911F9108958FE99FE06B
:102100000197F1F700C000002197F0CF811531F061
:1021100090918704892B809387040ACF08958115B5
:1021200019F00E94BC0504CF0895EF92FF920F931F
:102130001F93CF93DF93C62FD42F122F811599F0C1
:10214000609379040ADC9093140280931302C770A1
:1021500081E001C0880FCA95EAF7D8DFCDB7DEB7B6
:10216000E6E00C9444328091790468132FC0E0902B
:102170001302F0901402F1DB8E199F09883C91053F
:1021800028F500E20D0FCD1799F0C770FF24F394E6
:102190008F2D01C0880FCA95EAF7C1DF083040F4DF
:1021A0008D2F877001C0FF0C8A95EAF78F2DAEDF67
:1021B00060E070E0812F94DF083080F6D77081E016
:1021C00001C0880FDA95EAF7AADFC8CFC77081E0AF
:1021D00001C0880FCA95EAF7F7CF811531F09091C9
:1021E0008904892B80938904A3CE0895811539F041
:1021F00080959091890489238093890499CE0895CC
:1022000080917504811521F082E2F0DF109275044F
:10221000089510928704809120018130A1F480916B
:10222000400587FF10C0E2EFF1E08EE1DF011D9273
:102230008A95E9F780E090E0DDDA80E090E002DB6B
:102240001092890475CEEAEEF1E086E0EFCFE1DF8F
:102250002FEF84E39CE0215080409040E1F700C0E4
:10226000000088E19CE00FB6F894A8958093600088
:102270000FBE90936000FFCFAAE2B0E0E2E4F1E18C
:102280000C942B3288E192E0FC0101962091F10040
:10229000208322E080329207B9F7809119028930B9
:1022A00009F457C0C8F4823009F4B2C0833009F48D
:1022B00082C0813081F18091E80083FFE6C0809187
:1022C0001802909119029A3008F0DFC0E92FF0E06F
:1022D000E353FC4C0C94F3318A3009F489C08B3001
:1022E00051F780911802813231F780911C02909150
:1022F0001D02892B01F78091E800877F8093E80019
:1023000001DC81E090911A02911101C080E080937C
:1023100020017FDFD0CF80911802813A61F6809151
:10232000E800877F8093E80080911C0290911D0255
:10233000892B59F060E080E090E070E08ADB8091CA
:10234000E8008B778093E800B6CF68E080E292E007
:10235000F4CF80911802813209F0ADCF80911C0238
:1023600090911D028D7F892B09F0A5CF8091E80007
:10237000877F8093E8008091E80082FF17C09091EA
:10238000F3008091F200029731F48091F1008130E6
:1023900011F0863021F48091F10080931F0180912B
:1023A000E8008B778093E800ADDB85CF80917203E6
:1023B0008111E1CF80CF80911802813A09F07BCF63
:1023C00080911C0290911D02892B09F074CF80919D
:1023D000E800877F8093E8008091E80080FFFCCFD1
:1023E000809120018093F1008091E8008E77DACF10
:1023F00080911802813209F05ECF8091E800877FDA
:102400008093E8007FDB80911B0280931E0153CFF5
:1024100080911802813A09F04ECF8091E800877FC1
:102420008093E8008091E80080FFFCCF80911E013E
:10243000D9CF803889F0823841F580911C028F70A5
:10244000873018F58093E9008091EB0085FB8827A1
:1024500080F91092E90006C080914F03880F909197
:102460001502892B9091E800977F9093E800809364
:10247000F1001092F1008091E8008E7723C0811165
:1024800016C080911A02813009F18091E80083FF23
:102490000AC08091E800877F8093E8008091EB007C
:1024A00080628093EB00AA96E3E00C94473282307E
:1024B00061F780911A02811581F01092E9008091F4
:1024C000E800877F8093E8001DDBDFCF81E0933059
:1024D00009F080E080934F03F0CF80911C028F7051
:1024E0002FEF280F263088F68093E9002091EB002B
:1024F00020FFE3CF933031F48091EB008062809332
:10250000EB00DBCF9091EB0090619093EB0021E02A
:1025100030E0A90102C0440F551F8A95E2F74093AD
:10252000EA001092EA008091EB008860E8CF811108
:10253000ACCF10911A021F778091E3008078812B35
:102540008093E3008091E800877F8093E800DADAE7
:102550008091E80080FFFCCF8091E3008068809349
:10256000E30083E0111101C082E0809372038DCFFC
:102570008058823008F089CF80911A0290911B0216
:102580008C3D53E0950791F583E08A838AE2898345
:102590004FB7F894DE01139620E03EE051E2E32FBE
:1025A000F0E050935700849120FF03C082958F7014
:1025B0003F5F8F708A30C0F0895C90E08D939D936F
:1025C0002F5F243161F74FBF8091E800877F8093B0
:1025D000E8006AE270E0CE0101963BDA8091E80003
:1025E0008B778093E80051CF805DE7CF292F332789
:1025F0002330310509F44EC078F52130310509F456
:1026000088C08BE590E0EFE2F2E02230310509F07E
:102610003CCF2091E800277F2093E80020911E0204
:1026200030911F028217930708F49C0140E02115A6
:10263000310509F073C0411171C08091E80082FD3D
:10264000CDCF80917203811549F2853039F28091A6
:10265000E80083FFF2CFC2CF80911C0290911D024F
:102660002132310509F446C02232310509F00DCF7F
:102670008330910508F009CFFC01EE0FFF1FE15DEB
:10268000FE4F0190F081E02D845D9E4FDC018C9126
:1026900090E010C09C013327823021F123303105B6
:1026A00068F4232BB9F4ECEEF2E0E4918E2F90E085
:1026B000ECEEF2E0009709F4E8CEABCF2330310521
:1026C00009F0E3CEECE9F2E0E4918E2F90E0ECE942
:1026D000F2E0F0CFE2EDF2E0E4918E2F90E0E2ED57
:1026E000F2E0E8CFEAEBF2E0E4918E2F90E0EAEB43
:1026F000F2E0E0CF8330910508F0C7CEFC01EE0F89
:10270000FF1FEB5CFE4F0190F081E02D89E090E02F
:1027100080CF82E190E0EAE8F2E07BCF8091720323
:10272000811509F45BCF853009F458CF8091E8001A
:1027300083FD54CF8091E80082FD7FCF8091E80037
:1027400080FF75CF9091F3008091F2002115310543
:1027500019F08830910550F041E0089709F040E009
:102760008091E8008E778093E80061CF4491409398
:10277000F1003196215031090196E8CF803809F0F7
:1027800084CE8091E800877F8093E80080911602D4
:102790008093F10070CE811178CE10911A02123020
:1027A00008F073CE8091E800877F8093E800109353
:1027B0001602A8D91115D9F084E08093720342E083
:1027C00061EC81E01CDA42E261EC84E018DA42E27A
:1027D00061EC82E014DA42E260EC83E010DA80918E
:1027E0007203843051F482E0809321014ECE8091B7
:1027F000E30087FDE1CF81E0E0CF81E0F5CF86E027
:1028000090E00E9418338093740482FD06C085E333
:102810008093740484E794E05EDB809174048833D1
:1028200020F0877080638093740490917404892FE2
:10283000817090FF04C0892F8695869586950C94AB
:10284000720A0F931F93CF93DF93843030F5653076
:1028500020F54F3010F5C42FD0E0CC0FDD1F2EE156
:10286000629FC00DD11D112436E9839FC00DD11D7B
:102870001124CE0189960E941833082F10E0102FE2
:102880000027CE018A960E9418339801282BC9018F
:10289000DF91CF911F910F91089580E090E0F8CFE4
:1028A000462F672F2091750330917603232B81F4F7
:1028B000703F39F4403F61F4809173039091740349
:1028C0000895753028F44F3018F4843008F4B9CFE7
:1028D00080E090E00895A0E0B0E0E1E7F4E10C943E
:1028E00027327C0100913F0580913E05082BC3E013
:1028F000D0E010E0C8010C2E02C0959587950A948F
:10290000E2F780FD09C02197A8F7D12C8D2DCDB716
:10291000DEB7E7E00C944332DC2EB7018C2FC0DF2A
:102920000E94C206019779F3F1CF0F931F93CF93C3
:10293000FC0187819085009789F485810081118150
:10294000811581F0611571F0C801C5DFC82F682FAE
:10295000C8010E940E05B8018C2FA2DFCF911F91F4
:102960000F910895C8010E944405C82FF4CFCF935A
:10297000DF93D82FC92FAFDF6D2F7C2F91DF0E94FF
:10298000C206DF91CF910895FC0184818115B1F0D9
:10299000878190850097A1F00E94C206282F92950A
:1029A0009F709630B9F080F4925F9F70923030F44F
:1029B000203FD1F058F481E0283E58F080E008959F
:1029C00080819181D4DFEACF9A5FEFCF81E0243F0D
:1029D000A9F7089591E0813F09F090E081E0283E59
:1029E00008F080E0892B089581E00895382F292F81
:1029F000CB01A32FB22F8F3F9105A105B10520F484
:102A00008F5F9C4F0C94183380E0089585E290E02E
:102A10000E9418338A3889F486E290E00E941833C5
:102A20008F3259F487E290E00E94183391E08B36A0
:102A300009F090E0892F8170089580E0FCCFA0E03C
:102A4000B0E0E5E2F5E10C942532EC0188818115D6
:102A500009F1813009F045C08981813051F48A81C2
:102A6000239660E570E0893311F060E070E038DBB8
:102A7000EDCF823021F48A812396AEDAE7CF83301E
:102A800021F48A81239608DBE1CF843041F022963D
:102A90008111DCCFCDB7DEB7E9E00C9441328A81F9
:102AA000239620E030E09AE0682F6053770BAB016B
:102AB0006A30710560F02115310551F3EFE9FFE04F
:102AC0003197F1F700C0000021503109F4CF929FF7
:102AD000B001939F700D11249A01260F371F899121
:102AE000E3CFE82FF0E0E155FE4FB490282F269574
:102AF0002695269530E0F901E156FE4FE490877067
:102B0000F12C082E02C0F594E7940A94E2F7E0FA5B
:102B1000EE24FF24E0F8F901E157FE4FC490D12CD8
:102B2000082E02C0D594C7940A94E2F7C0FACC24C8
:102B3000DD24C0F8F901E158FE4F049110E002C015
:102B4000159507958A95E2F701701127E114F104B4
:102B500011F081EE41DAC114D10411F086EE3CDAB5
:102B600060E070E08B2DBCDAC114D10411F086EE68
:102B700093DAE114F10411F081EE8EDA01151105FA
:102B800021F060E070E08CE2ABDA21965FCFAAE042
:102B9000B0E0EDECF5E10C942632E9E7F2E080E5F7
:102BA000DF011D928A95E9F7EFE8F4E088E3DF01A1
:102BB0001D928A95E9F789E7C82E82E0D82E7F0119
:102BC00001E812E0F701D182C0824AE050E0B8018A
:102BD000CE0101960E94083388E0FE013196D601AD
:102BE00001900D928A95E1F789859A85D701139610
:102BF0009C938E931297BAE0CB0ED11CE7E0EE0EB9
:102C0000F11C065F1F4F013DF2E01F07D9F62A961F
:102C1000E8E00C944232A6E0B0E0E1E1F6E10C9489
:102C200027320EE114E081EDE82E82E0F82E98E0E4
:102C3000D92E46E050E0B701CE0101960E9408333C
:102C4000F8018D2D11928A95E9F7B8016C5F7F4FDD
:102C500089819A810E94190BF80191838083B801C0
:102C60006B5F7F4F8B819C810E94190BF8019383CE
:102C700082838D8186838E818783F6E0EF0EF11C3F
:102C8000085F1F4F81E0E81683E0F80691F626966C
:102C9000E7E00C944332AAE0B0E0E1E5F6E10C9401
:102CA0002132C0907003D090710381E090E0909346
:102CB000710380937003812C912C10E0540100E08B
:102CC00019C021E030E0123020F4F7018591959190
:102CD0009C01472D602F812F04D9739422E0E20ECE
:102CE000F11C3FE07312EDCF0F5F8FE0A80EB11C17
:102CF000053049F0C501880F991FFC01E051FD4FD7
:102D00007F01712CDECF1F5FFBE48F0E911C14300E
:102D1000A9F69E012F5F3F4F79018AE0F9011192D8
:102D20008A95E9F701E812E04AE050E0B801C701EE
:102D30000E945733065F1F4F013DF2E01F07A1F7C6
:102D400086E0F70111928A95E9F746E050E0B80174
:102D5000C7010E9457330A5F1F4F0130F3E01F077E
:102D6000A1F7D0927103C09270032A96EDE00C9403
:102D70003D32A0E0B0E0EFEBF6E10C942032FC0134
:102D80008280648081E08483ECE1F4E09490EBE95C
:102D9000F4E0E491009180040695015810E0000FE2
:102DA000111F012F1127C9ECD2E0C12CD12CAA246C
:102DB000AA94B12C77247A94E919EE2EF12C83E0B1
:102DC000881630F480917E04888380917F04898303
:102DD000611017C01B821A8296014A81698188811D
:102DE0000E9461088FEFC81AD80A259688E1C81694
:102DF000D10429F70E947D08CDB7DEB7EEE00C9430
:102E00003C328B818115E9F081508B83789EC00123
:102E100011246C8170E00E94CC31FB01FF27E45E3D
:102E2000FB4F8491E82FE9197E9EC0011124B70160
:102E30000E94CC3180918004689FB00111247A8374
:102E4000CBCF0E94D032B5010E94E03180179107AC
:102E50001CF683E0881688F00E94D032B5010E94EB
:102E6000E03188830E94D03220917F042695622F22
:102E700070E00E94E031280F29831A82809180043B
:102E8000893C20F088EC8C838B83A6CF8431D8F7E3
:102E900084E1F9CF0F93CF93DF93CDE7D4E048815E
:102EA00059816A817B8188E090E00E944B332881C0
:102EB00039814A815B816C817D818E819F8100E2B5
:102EC0000E946E32622F83E290E00E943933DF91DC
:102ED000CF910F910895EDE7F4E085E080831182B2
:102EE0008FEF828383831482CF01D4CF80918104BA
:102EF000833018F48F5F809381048DE794E0CACF0C
:102F000080918104811519F08150809381048DE7AF
:102F100094E0C0CFA0E0B0E0E0E9F7E10C9421320A
:102F2000182FF62E042FE22E90917D0490FF23C0DF
:102F3000E92FE695E695AE2FB0E0A55CBE4F8C91EB
:102F400080937B049C7F9430D9F4612F7F2D842F54
:102F50000E94DA07962F672F482F892F0E94920828
:102F600010937E04F0927F0400938004E11419F022
:102F70008DE794E08FDFCDB7DEB7EDE00C943D3206
:102F8000823019F400918004EBCF863019F410914F
:102F90007E04E6CF8930D9F3893111F7E9518E2FBC
:102FA0008170782EE695F0E0E45EFA4FE491CE2F42
:102FB000D0E0A12CB12CC12CD12C88E1882E912CF1
:102FC000C501B4010E94CC31812F711012C0860F4F
:102FD0009601402F6F2D0E9461088FEFC81AD80A02
:102FE000AC0EBD1E88E1C816D10451F70E947D08C1
:102FF000B7CF861BEDCFEDE7F4E0818121E043817F
:103000006281885F87CFEDE7F4E0818121E0438131
:10301000628188507FCFEDE7F4E0628121E1620FA9
:1030200008F46FEF21E04381818174CFEDE7F4E094
:10303000628121E1621B08F460E021E0438181812B
:1030400069CFEDE7F4E0438121E1420F08F44FEF4F
:1030500021E0628181815ECFEDE7F4E0438121E1EF
:10306000421B08F440E021E06281818153CF9091BE
:103070007D0490FF2CC0811559F18B3258F58F7368
:10308000880F880F90917D049370892B80937D0425
:10309000611519F08DE794E0FDDE60917D04669581
:1030A000669570E04BE050E087E091E00E94E732E7
:1030B000892B91F010927C0481E080935E0320E0E4
:1030C0004091800460917F0480917E0423CF089515
:1030D00081E0D6CF8AE2D4CF81E080937C040E9445
:1030E000AD0C90935C0380935B03E6CF80917D04ED
:1030F000869586958F5F8B3208F081E061E0B7CFCF
:1031000080917D04869586958A9509F48AE261E02E
:10311000AECFA9E0B0E0EFE8F8E10C941C328C01EE
:10312000DC0114968C91811509F4A9C061E0C801F5
:10313000FCDB7C0180917304811135C0F80185812D
:10314000811509F450C0E114F0E5FF06B8F5E1146B
:1031500020E2F20608F097C0E11437E0F30619F117
:10316000F0F4C701805E91090897E8F03091870478
:10317000809189042091860499E0F801AFE5B4E0DC
:1031800001900D929A95E1F7F0926704E09266043F
:1031900010926904832B822B80935E0404C0E11497
:1031A0005FE0F50619F7F801458141116EC133E77B
:1031B000E3163CE7F30609F05FC251C090EEE91652
:1031C00092E5F90650F4A0E6EA16A2E5FA0658F7E9
:1031D000C701925580349105C8CF970127573C47C6
:1031E0002530310518F6F9E7EF16FCE7FF0609F080
:1031F0004EC02091660430916704232B81F1811524
:10320000A1F081E00E94C50B80915E040E94ED1048
:1032100089E0EFE5F4E0A5E1B4E001900D928A9534
:10322000E1F7809169048093140486E0F801A5E138
:10323000B4E001900D928A95E1F780911404809397
:10324000730485E194E065DF10927304D80115964C
:103250008C91811104C080915E040E94F6108091CF
:103260008A048770811559F0F8018581811539F03C
:103270008091410582FF03C082E00E94A10529964A
:10328000E2E10C943832F801868180316ECFBAE7E2
:10329000EB16BCE7FB0609F086CF811509F4CAC01E
:1032A000A0906604B0906704E0915E04E887E9832B
:1032B000BE016F5F7F4FC5010E94190B2C01F98180
:1032C000F987FEE1CF2EF4E0DF2EEE24E394F12C1B
:1032D00022242A94D60117963C90179733FE54C0A7
:1032E0006D907C90119712968D909C901397461438
:1032F0005704B9F41496BC91BF83232DF60146817F
:103300006B2F89850E94330B811559F08F810E94A4
:10331000D404281634F4D60115969C917401F92A28
:10332000282E48145904C9F431FE17C0F601F5815E
:10333000FF83232DD60116964C916F2F89850E940D
:10334000330B811551F08F810E94D40428162CF480
:10335000F60194817301F92A282E30FE15C0FFEF83
:103360002F1212C021E0E216F10471F4232DD601D0
:1033700016964C9160E089850E94330B811521F0EF
:10338000F60185817401F82AF8E0CF0ED11C2EE5F4
:1033900034E02C153D0509F09DCF31E0E316F10432
:1033A000F1F5988592959F704885942B9F7081E0E8
:1033B000403108F480E0F82EF294E0EFFE22F92A82
:1033C000A11450E2B50620F5A11481E0B80608F07A
:1033D00055C0EA2C8F2D8D704A2D811509F451C0EE
:1033E0006AE084ED98E00E94D60B282F30E021158A
:1033F000310551F44E2D66E186EB98E00E94D60B24
:10340000282F30E0811549F0F901FF297F0107C01D
:10341000C50190528115904390F1E12CF12C87E089
:10342000EAE6F4E0DF011D928A95E9F7F092720472
:10343000E09271048091710490917204892B09F4D7
:103440000ECFF8018581811539F08FEF0E94C50BF1
:10345000809169048093680486E0F801AAE6B4E0EC
:1034600001900D928A95E1F780916804809373042E
:103470008AE694E04EDE10927304F1CEFB28BB2462
:10348000A8CF68E08CEC98E0AECFC70197578038A2
:10349000910508F0DAC0BE2CF0E1EF1608F0DFCE9F
:1034A0006EEF70E080E090E0A1DA8111D8CEC12CFF
:1034B000D12C7601B11044C074E0272EAE014F5FCD
:1034C0005F4F5E834D83AD81BE81E22D1D92EA95F3
:1034D000E9F746015701FFEF8F1A9F0AAF0ABF0AAB
:1034E000C701B60183DA8983811509F4B8CE81302A
:1034F00009F0A7C02601370122E0420E511C611CD1
:10350000711CC501B40172DA382E8A83811509F461
:10351000A6CE8FEF830D833030F5C301B20166DA9A
:103520008B83811519F0CE01019689DA4601570186
:1035300033E0830E911CA11CB11C75016401C3CF43
:103540002FEFC216D104E104F10409F488CEC701BB
:10355000B6014CDA3FEFC31AD30AE30AF30A81112A
:10356000EFCFBA94A7CF8BEF830D8330A8F5460138
:10357000570143E0840E911CA11CB11CC301B20190
:1035800035DA8B838115C9F2C501B4012FDA8C833A
:10359000811108C04601570154E0850E911CA11C01
:1035A000B11CCBCFAB80BC8081E0A8168FEFB806F2
:1035B00010F0BA2CAA2496E0391651F0A7E03A167A
:1035C00019F0C5010E944E27C5010E948027E2CF55
:1035D000C5010E944E27DECFB4E0530142013B12E9
:1035E000ACCFC301B20102DA782E46015701E4E004
:1035F0008E0E911CA11CB11CC701B6016D5F7F4FDF
:103600008F4F9F4FF3D9711409F429CE811509F416
:1036100026CE8150990B4FEF489F9001499F300D66
:103620001124472D4150550B240F351F21503109CE
:1036300008F483CF8FE99FE00197F1F700C0000005
:10364000F5CFCE010196FBD978CFA3E0EA16A8E723
:10365000FA0609F44CC058F5E1E0EE16E8E7FE067C
:10366000F1F1F2E0EF16F8E7FF0609F471C086E029
:10367000E11428E7F206A1F182EAE81682E5F806ED
:1036800009F4C4C093EAE91692E5F90608F096C079
:10369000C70190528115904208F4ABC0F1EEEF16CD
:1036A000F10409F4B3C025EEE216F1048BC034E056
:1036B000E31638E7F306C1F155E0E51658E7F506DD
:1036C00009F45AC053E7E5165CE7F506D9F6809190
:1036D0007504811509F462C00E940011C0CD80E01C
:1036E0000E94040B84E794E00E946B0FB8CD809198
:1036F0007404883088F088508093740491E0883096
:1037000008F490E08091740490FB80F98093740435
:1037100084E794E00E946B0F8091740486958695EF
:1037200086950E94720A9BCD90917404892F86958C
:1037300086958695903340F48F5F880F880F880FA9
:103740009770892B80937404809174048160DECF1C
:103750008091740480FF09C08E7F8093740484E795
:1037600094E00E946B0F80E0DCCF81608093740452
:10377000813071F689E0CACF809174048695869570
:1037800086958F5F8F71873008F080E0880F880FF3
:10379000880F909174049770892BAECF1092870494
:1037A0000E94C4050E94AD0C88579C4E90937704EC
:1037B0008093760481E08093750451CDB2EBEB16D3
:1037C000B2E5FB06E1F525EE30E02770332781E016
:1037D00090E001C0880F2A95EAF720917804309193
:1037E00075043115D9F04115A1F0282B20937804E8
:1037F00036CDF8018681803110F58F2D99278F7194
:1038000099278230910511F04297DCCF21EE30E00C
:10381000DCCF809582238093780421CD322F38230A
:10382000311569F0982F90959223909378040E9417
:10383000BC05D80115968C91811509F410CD8091A5
:103840007504811509F4D1C0C0908704D090860416
:103850000E94AD0C88579C4E909377048093760419
:10386000F8018581811509F4C0C08D2D8C298D79D1
:10387000811190C0E114F0E5FF0608F5E11420E4A1
:10388000F20608F09BC036EEE316F10409F449C0D5
:10389000C70190528115904208F097C0D801169642
:1038A0008C91803108F46EC0C70199271092890469
:1038B0008D32910509F582E0809389048AC0B0EECB
:1038C000EB16B2E5FB0608F04DC0E0ECEE16E2E5C3
:1038D000FE0638F5F0EAEF16F2E5FF06E8F420E61A
:1038E000E21622E5F206E8F4C7019255803491050C
:1038F000C0F010928904C7018E32910508F082C091
:103900008832910508F063C08E31910508F061C0DE
:1039100004974A9780F23EC034EBE31632E5F30693
:1039200041F7D80115969C91911509F44DC5109257
:103930007904970130572332310508F02CC584E013
:1039400090E00E9425339093410580934005F70154
:10395000E150F047E232F10508F077C0E952FC4C43
:103960000C94F33149E7E4164CE7F40630F457E7DA
:10397000E5165CE7F506A8F6BCCF8BE7E8168CE702
:10398000F806CECF8F2D8F71843159F2863161F4D4
:10399000109289040E94001180918704909178040C
:1039A000892B8093870421C00E9400118091870495
:1039B00090917804892B80938704B3CFD801169611
:1039C0008C91803108F070CFACCFC7016FCF8A9750
:1039D00009F780917804811531F08091890492E093
:1039E0008927809389040E94980FF8018581F70147
:1039F000E851FC47E730F10508F093CFE750FC4C65
:103A00000C94F3318C34910521F38D329240E0CF48
:103A100026E241EE61EE0E94951021CC27E245EEB0
:103A200065EEF9CF26E241EE60EEF5CF27E245EEF6
:103A300064EEF1CF26E241EE62EEEDCF27E245EEF5
:103A400066EEE9CF28E241E0EBCF8091400581604E
:103A500080934005609140057091410584E090E0BD
:103A60000E9453330E940911FACB8091410588606E
:103A700080934105EFCF809140058260E9CF80912E
:103A800040058460E5CF809140058860E1CF80915A
:103A900041058160EDCF809141058260E9CF809141
:103AA00040058061D5CF809140058062D1CF809163
:103AB00040058064CDCF0E94091180914005806847
:103AC000C7CF809140058C60C3CF80914105836052
:103AD000CFCF809140058E7FBBCF80914105877FFE
:103AE000C7CF809140058D7FB3CF809140058B7FFC
:103AF000AFCF80914005877FABCF809141058E7F0E
:103B0000B7CF809141058D7FB3CF809140058F7EE7
:103B10009FCF809140058F7D9BCF809140058F7B0B
:103B200097CF0E940911809140058F7791CF8091A6
:103B30004005837F8DCF809141058C7F99CF809107
:103B40004005992782FF939590FB82F990FB83F9BA
:103B50007FCF80914105982F909590FB80F990FB45
:103B600081F986CF90914005892F8F7B96FF8064E5
:103B70006FCF0E94091190914005892F97FB87F91B
:103B8000805866CF61E08EE090E00E94393362CFCA
:103B900060E0F9CF90914005892F8F7E94FF80617E
:103BA00057CF90914005892F8E7F90FF816050CF35
:103BB00090914105892F877F93FF886059CF89E2D3
:103BC000FDC389E20DC48272F701E052F847EB3081
:103BD000F10508F04DC0E050FC4C0C94F331B7E710
:103BE000EB16BCE7FB0609F048C081E00E94000527
:103BF00068C080917D0480FF0BC08E7F80937D0420
:103C00008DE794E047D910927C040E947D0827CB71
:103C1000816080937D0461E08695869528DA1FCBCC
:103C2000811521F06DDA1BCB8115E1F35FDA17CB3B
:103C3000811521F0E8D913CB8115E1F3DCD90FCB45
:103C4000811521F0F3D90BCB8115E1F3E4D907CB32
:103C5000811521F001DA03CB8115E1F3F2D9FFCA16
:103C6000811521F04DD9FBCA8115E1F33FD9F7CA7F
:103C7000E7E7EE16ECE7FE0609F1F8E7EF16FCE7DA
:103C8000FF0629F19701205E32452032310520F5EB
:103C9000911122C02E2D2F7181E090E0AC0102C065
:103CA000440F551F2A95E2F77A01642F83E090E0D4
:103CB0000E9439338E2D0E94F004D1CA81E00E9407
:103CC000F60443E062E081E00E947805C8CA82E021
:103CD000911509F48BCFF3CF4091850480913F0576
:103CE000282F30E02095309570E024233723232BB4
:103CF00019F04823409385045BE7E5165CE7F50679
:103D000041F4911509F4ABCA0E94D7040E949E0B9E
:103D1000A6CA80E4E81682E5F80608F05AC0A0E2D8
:103D2000EA16A2E5FA0608F05BC0E114B0E5FB066E
:103D300070F5E114E0E4FE0608F068C0911509F49E
:103D40007EC0BAE5EB16BCE7FB0609F4F5C008F047
:103D5000D7C0F1E0EF16FCE7FF0609F4EBC023E063
:103D6000E2162CE7F20609F4DFC0E1143CE7F306A3
:103D700009F065C00E9409118FEF94E3ACE0815017
:103D80009040A040E1F700C000000E94CE0E9701D5
:103D900030552115324090F6970145E0369527952C
:103DA0004A95E1F7822F8F702091850430E041E041
:103DB00050E0082E02C0440F551F0A94E2F7242356
:103DC0003523232B09F4BACF9111A0CF1092870489
:103DD000F7C29701205C32452032310508F0AECFA2
:103DE0008E2D8F712091850430E041E050E0082E47
:103DF00002C0440F551F0A94E2F724233523232BD6
:103E000009F49CCF911509F42ACA80CFD8011696DF
:103E10008C91803108F092CF911111C02F2D2F700D
:103E200081E090E002C0880F991F2A95E2F7209167
:103E3000850430E082239323892B09F010CAD8012E
:103E400017968D919C91009709F47AC00E94C20642
:103E5000D82EF92ED8011596BC9015971696AC90D1
:103E6000A2942FE0A22280918A048770811509F123
:103E7000CB2CB114F9F0892F807F803469F080E277
:103E80008D0D8830B0F0892F807E803229F4B2E029
:103E9000DB1678F0A11469F08091410582FF09C01A
:103EA00082E00E94A10580918A048770CC24C3948B
:103EB0008111C12C8F2D82958F70883009F463C1D8
:103EC00008F072C0843008F053C0EF2DEF70EE2E72
:103ED000823008F47AC08F2D807F803219F0E2940E
:103EE00080EFE822D11409F4A8C031E0D31609F418
:103EF0000CC1B11409F418C1A11409F4BCC07CC0F0
:103F00004BE5E4164CE7F406C9F080914105002426
:103F100082FF0394802D5CE5E5165CE7F50609F069
:103F20008ECF0E94540F8BCF6FEF7FEF80E090E039
:103F30000E9453330E94271181E0F3CF80E0F1CF3C
:103F4000F8018581C080D180811569F0C6010E9489
:103F50006B14F82E682FC6010E940E05B6018F2D36
:103F60000E94501473CFC6010E944405F82EF6CF6C
:103F7000843009F4EBC0C11409F437C180918A047C
:103F800080FD33C1D80115961C928695869586953D
:103F90000E94F604C801BDD880918A048695869552
:103FA00086950E94000521C1893009F463C18A5FAA
:103FB0008F70823000F7F2EFDF126FC18F2D8F719B
:103FC000B11068C10E94F6040CC120E1F21618F08D
:103FD000E29490EFE922B114B9F0E11469F080E2C3
:103FE0008D0D883010F0D11009C0809187048E2982
:103FF000809387040E94980F8D2D2FC08091890493
:104000008E2980938904F6CF8D2D0E944C10E114E7
:1040100009F4B1CF80E28D0D883010F0D11004C0CA
:104020008E2D0E94BC0506C0E094809189048E21EB
:10403000809389040E94980F9ECF8091410582FD54
:1040400016C0B11469F0E11439F0809187048E290B
:10405000809387040E94980F80E00E94EC0F8BCF22
:1040600080E00E944C10E11409F485CFD9CFB1143F
:1040700071F1A11004C08E2D0E9486107CCF41E00A
:10408000A41211C0F09086048E2D8F21E81609F439
:1040900072CF0E94AD0C90938E0480938D04FE2805
:1040A000F092860468CF55E0A51265CF8E2D0E9450
:1040B00086108E2D0E94070D809188049E2D9823D6
:1040C000E91609F458CF8E298093880454CFA110A3
:1040D00012C08E2D0E948F108E2D0E94070D809190
:1040E00088049E2D9823911509F445CFE094E82289
:1040F000E092880440CF81E0A8123DCF80918704F0
:104100008E21811509F437CFE4CFB11429F096E060
:10411000A91608F030CFAFCFA5E0AA1608F02BCF34
:104120008E2D0E948F1027CFA114D1F3B9E3DB129B
:1041300009C0EFEFF7EE23E0E150F0402040E1F757
:1041400000C000008D2D0E944C1015CF8F2D86953C
:1041500086958370811569F0813009F00CCF8D2D23
:104160009F2D9370B11002C080E090E00E94220C5D
:1041700002CF8D2D9F2D9370B11002C080E090E092
:104180000E94FA0BF8CE8F2D837081113BC0B110C5
:1041900028C04D2D429546954770440F440F8D2DF4
:1041A0008F70042E01C0880F0A94EAF72D2D20711C
:1041B000D4FE07C02FE030E001C0220F4A95EAF795
:1041C00020953F2D3695369533703230B1F033302F
:1041D00091F040913E05313069F0822B84230E949A
:1041E000F0040E94EB0B0E94EA0460E0C8010E9408
:1041F000951445C8842B822BF2CF822B90913E05DB
:104200008927EDCFB11459F1F0FEEBCF4D2D42953A
:1042100046954770440F440F8D2D8F70042E01C0BA
:10422000880F0A94EAF72D2D2071D4FE07C02FE0E5
:1042300030E001C0220F4A95EAF720953F2D3695D0
:1042400036953370323089F0333069F040913F0554
:10425000313041F0822B84230E94F304C2CF82309C
:10426000A8F6BFCF842B822BF7CF822B90913F05EE
:104270008927F2CF3F2D3F70F32EB11439F0832FF1
:104280000E94F6048D2D0E948610ABCF8D2D0E94CA
:104290008F108F2D0E940005A4CF43EFD41680F419
:1042A00050EFD516E1F081EFD816A1F0B11409F462
:1042B00060C0A11409F45AC08D2D0E94EC0F91CF5B
:1042C00093EFD916F1F0A4EFDA12F0CF8091410507
:1042D00082FD23C08F2D8F71B114E1F273CEB11422
:1042E00069F0B5E0AB1608F07CCF2F2D2F7181E07F
:1042F00090E001C0880F2A95EAF7B8CFE6E0AE1645
:10430000F2CF80E0B11409F4A7CF9F2D9F7181E017
:1043100001C0880F9A95EAF79FCFB114C1F0809140
:104320008A048770843049F410928A0410928C04B5
:1043300010928B048F2D8F71ADCFF5E063E0AF1637
:1043400008F04FCF8F2D8F710E94F10C4ACF25E0DE
:10435000A21640F010928A0410928C0410928B04E2
:1043600064E0F0CF81E00E94A1053BCF8F2D8F71DB
:1043700029CEA114F9F239E3D31209C04FEF57EE59
:1043800083E0415050408040E1F700C000008D2D97
:104390000E944C1026CF80918704F6E1EF16FCE7CF
:1043A000FF0609F010CC8A7A91E0811101C090E0FB
:1043B00090937A04811509F402CC85E30E944A0C9B
:1043C0000E94980F0C942F1926E1E2162CE7F206B2
:1043D00009F005CC80917A04811509F4F2CB85E3CC
:1043E0000E947E0CEDCF8091F303803178F48091B0
:1043F000F203811559F0E091A4032091A3033091B9
:10440000EE034091ED0359E02E1301C008956E2F85
:1044100070E05E9FF0011124DF01AB55BC4F149694
:104420008C911497811559F111968C9111978313E2
:1044300026C08C91841323C015968C9115978111F9
:104440001EC012968D919C91A091EF03B091F00344
:104450008A1B9B0B883C910590F48091F3038F702D
:1044600080618093F303E555FC4F80818F708061FC
:1044700080838DEE93E00E9489180C949705FB01D0
:104480003196E770C1CFAFE0B0E0E9E4F2E20C941E
:1044900020328C0186E0F801DE011A9601900D921F
:1044A0008A95E1F7F801F58084819DEE892E93E0ED
:1044B000992E6090F103611017C0811591F0F114ED
:1044C00009F43FC1C8010E94C414811509F439C11F
:1044D00089E0F801ADEEB3E001900D928A95E1F725
:1044E00082DFFF24F3945FC07080A280B380D090FD
:1044F000F2032091EF033091F003A501421B530B0F
:10450000D11409F4E5C0483C510508F08CC0811570
:1045100041F38091EE03C180E090F30350E1E51692
:1045200008F062C0C8121EC08091ED0387111AC046
:104530002091F4033091F50387819085281739077E
:1045400089F4F1104BC08E2D8F7080618093F3033E
:104550008DEE93E00E9489188091F303F801868321
:10456000F12C21C0F1103AC040E06C2D872D0E9443
:10457000890E40E06C2D872D0E94890EF82E811146
:10458000EFCF8A859B850E94B714292F22952F7023
:10459000903470F49F702230A0F09115B1F0F801C2
:1045A0009681903190F48F2D2F96EEE00C943C3252
:1045B0002A5F2F70223068F0C8010E948918FD2CF4
:1045C000F2CF911511F0811571F3805E883058F3A8
:1045D000F3CF803F40F3815F8330F9CF8091F303C5
:1045E00081608093F303BCCFC8124EC08091ED036D
:1045F00087114AC02091F4033091F503878190859B
:104600002817390709F040C0F1103EC0E682C80102
:104610000E94891889E0F801ADEEB3E001900D9297
:104620008A95E1F75ECFE090F303F0E1EF1650F4E6
:104630008DEE93E00E94891889E0F40111928A9529
:10464000E9F78ECF811509F44CCF9091EE03F80174
:104650008181981319C08091ED03871115C02091B5
:10466000F4033091F503878190852817390761F4A9
:10467000F1100AC0E682C8010E94891889E0F4019D
:1046800011928A95E9F72DCFC8010E94C4148115B3
:1046900009F457C0F11409F454C08091F303803237
:1046A00008F416CF8091ED039091EE039A838983ED
:1046B000BC82AB826D821E82EF828091F403909166
:1046C000F50399878887CE0101960E94891800CF4B
:1046D000483C510508F0B0CF811509F402CFF11420
:1046E00081F19091EE038181981321C08091ED03B7
:1046F00087111DC02091F4033091F50387819085C7
:1047000028173907A1F48091F30380FD83CF80310E
:1047100008F480CF8683982F907F903F09F477CF5D
:10472000982F907F905F8F70892B868370CFC80100
:104730000E94C4148111CCCE8091F30381608093D8
:10474000F303C8010E948918CCCEA2E1B0E0EBEAE5
:10475000F3E20C942A320A871B872C873D874E8709
:104760005F87688B798B8A8BCE010A968CDE8111EC
:1047700028C02091A3033091A40389E0FE013A965A
:10478000DE01119601900D928A95E1F78E858115D3
:10479000C1F0822F90E0019687709927381719068B
:1047A000D9F099E0929FD0011124AB55BC4FFE0186
:1047B000319601900D929A95E1F78093A3030E94A0
:1047C000970519E08091A4039091A303891312C067
:1047D0006296E4E00C9446320E9409111092A30301
:1047E0001092A40389E0EDEEF3E0DF011D928A95BB
:1047F000E9F7E7CF189FC00111248B559C4F43DE8A
:10480000811531F38091A40390E001968770992778
:104810008093A403D7CFEF92FF920F931F93CF9370
:10482000DF9380913B05E0913002CDE0811130C0F3
:10483000CDB7DEB7E6E00C944432D1E0DE0FD09382
:104840003002EE2EF12CCE9FF0011124ED52FB4FE1
:1048500084818115E1F087819085892B21F4818500
:104860009285019651F40081118122813381448126
:10487000558166817781808568DFCE9DF001CF9D6F
:10488000F00D1124ED52FB4F148210928904ED2F8C
:1048900080913B05E81788F210923B051092300298
:1048A000C7CFA4E0B0E0E7E5F4E20C941D3220911C
:1048B000D204298397E0992E01E010E02DE0322EFA
:1048C00034E0532E882483948091D10499818913F4
:1048D00007C0A1DF0E94610B2496E1E10C943932FC
:1048E0009981892F90E09C838B83FC01EE0FFF1F41
:1048F000E953FB4F80819181989ED001999EB00D24
:104900001124FD01E157FB4FFA83E9832481211132
:104910005BC060903B05E3EDF4E060E070E0712C7B
:10492000661508F04FC0A384B484A981BA81CD90E4
:10493000DC902FEF3FEF412C442D50E07601E40C4A
:10494000F11CE40CF11CD701ED90FC90E114F10492
:1049500039F0AE14BF0409F0A90143949A01ECCFD9
:104960002F3F3207D1F1D80102C0AA0FBB1F2A95F1
:10497000E2F77A2A9801042C02C0220F331F0A940E
:10498000E2F7A901415051097416150629F5369E22
:10499000F001379EF00D1124ED52FB4F989ED0018F
:1049A000999EB00D1124A157BB4F12962D913C91A9
:1049B00013973087278354821082118292878187D0
:1049C00015968C920E94720B8B819C8101969A8322
:1049D00089838370898378CF14826F5F7F4F3D9680
:1049E0009FCF10923D0510923C05109222018091BC
:1049F000D1048093D2040E94610B0DCFACE1B0E0F2
:104A0000E4E0F5E20C941C324B8B5C8B6D8B7E8B5F
:104A10008F8BB92E988FA92E911110928904188A24
:104A2000198A1A8A86E0FE017396DE011A960190B1
:104A30000D928A95E1F75F888091410582FF1FC042
:104A40000E94AD0C20918B0430918C04821B930B3F
:104A50008838934138F080918A0482FD03C082E057
:104A60000E94A1050E94AD0C20918D0430918E040E
:104A7000821B930B8838934110F00E94C405511497
:104A8000D9F05E86BF8661E0CE010A960E94951439
:104A900061E0CE010A960E94951461E0CE010A966B
:104AA0000E9495144C0180356CE7960791F4A1148F
:104AB00019F181E0809322015E86BF860A851B85FD
:104AC0002C853D85452D5B2D688979898A893DDE58
:104AD000CDC081359C4721F4A11471F082DFECCF69
:104AE00082E588168CE7980639F4A11429F08091A4
:104AF00022018111F3CFDDCF4FE8E42E44E0F42E04
:104B0000412C612C712CD7016D917C91CC24CA94DD
:104B1000DD24DA9480E0282F30E0FB01E80FF11D5E
:104B2000E80FF11D408151814115510539F084167E
:104B3000950609F096018F5F6901EDCF10E0BFEF98
:104B4000CB16DB0609F44EC0F70144811091220117
:104B5000411110E0D70115963C90159716969C913F
:104B60001697A11409F405C1111509F402C13110F9
:104B700017C021E030E00C2C01C0220F0A94EAF7A4
:104B8000922B16969C932091CF043091D00422331F
:104B9000310530F422E330E03093D0042093CF0489
:104BA000E1E0F0E002C0EE0FFF1F8A95E2F7CF01CF
:104BB0000197D70116962C912817190699F4C090E1
:104BC0003C05D0903D05C114D10409F453C00E94A6
:104BD000AD0C8C199D09C39708F44CC081E0F70116
:104BE000848311E0412ABFEF6B1A7B0AE7E0EE0EE7
:104BF000F11CF8E06F16710409F085CFA11409F4D7
:104C000017C1411409F414C10E94AD0C90933D05E5
:104C100080933C0580913B05883040F591E0980FEA
:104C200090933B0599E0FE013A96DE0111960190C2
:104C30000D929A95E1F75D82BE822DE0829FC001C0
:104C400011248D529B4F29E0FE013196DC01019029
:104C50000D922A95E1F72FEF3FEFDC011A963C9376
:104C60002E9319971C969C928E921B976C96E2E15C
:104C70000C9438322091D2048091D104922FE0E03C
:104C8000F0E001E0281709F448C0422F50E0FA0193
:104C9000EE0FFF1FE953FB4F2080318037E0329D3C
:104CA000F001339DF00D1124E157FB4F60817181BC
:104CB0007C8F6B8FB0E030E0A0E0EB8DFC8DEA0FD5
:104CC000F11DEA0FF11DC080D180C114D104E1F0C3
:104CD000F7010190F081E02DFA8FE98F30E007C0F5
:104CE000E1E0C616D70609F0E0E0BE2B3F5FE98D94
:104CF000FA8DE30FF11DE30FF11D608171816115E4
:104D0000710571F7AF5FD9CFB11581F13A17C8F4CA
:104D1000E1E0D7011496EC93F7019093D204EE15DD
:104D2000FF0509F45FCF90E0FC01EE0FFF1FE95390
:104D3000FB4F718260820196837099278093D10422
:104D400051CF37E0329DF001339DF00D1124E15732
:104D5000FB4F0483EE15FF05F9F2291302C09F5F94
:104D600093709A012F5F3F4F23708CCFE0E0F0E00B
:104D7000F8CF292F30E0311024C061E070E002C08C
:104D8000660F771F8A95E2F7CB010197281739073D
:104D900091F010E0E1E0F0E002C0EE0FFF1FCA94D6
:104DA000E2F76F01C094D70116968C9116978C216B
:104DB00016968C9317CF411569F3C3010E94720BAD
:104DC000E8CFA9010C2C02C0559547950A94E2F74B
:104DD000C901019782239323892B39F540FF25C010
:104DE000D70112968D919C91892BD1F087E0FE011D
:104DF0003196DF011D928A95E9F70E94AD0C9C0166
:104E00008B839C8384E08D83F70192818381792F4A
:104E10009887898709811A8144E05E816F8195DCDA
:104E2000D70115961C92132DB5CF142F1170B2CF48
:104E30009091D2048091D104981731F032DDB1E025
:104E40004B1609F413CF38CEE6DC10923D051092D4
:104E50003C050E94610BF3CFA6E0B0E0E2E3F7E28D
:104E60000C942A320E94AD0C8C01809177039091B2
:104E700078038017910771F019821A820E94AD0C95
:104E8000BC0149815A8180E090E0B8DD109378033D
:104E9000009377032696E4E00C944632A6E0B0E057
:104EA000E4E5F7E20C942A328C019093740380932A
:104EB0007303011580E21807B0F4C801805E910900
:104EC000089728F06DEE70E10115110511F466E800
:104ED00070E1C8010E94A804802F0E94EC0F269662
:104EE000E4E00C94463280EF89838A830E94AD0C03
:104EF0008160BC0149815A8181E091E07FDDEFCF83
:104F0000A6E0B0E0E6E8F7E20C942A328C01909338
:104F1000740380937303011580E21807B0F4802FA7
:104F20000E944C10C801805E9109089728F066EF36
:104F300070E10115110511F46FE870E1C8010E94DC
:104F4000A8042696E4E00C94463280EF89838A8395
:104F50000E94AD0C8160BC0149815A8181E090E0E2
:104F60004DDDEFCFA0E1B0E0E8EBF7E20C941E32AC
:104F7000FE01319680E1DF011D928A95E9F700E19B
:104F800010E0AA24A39493E0B92E412C512C3201B5
:104F90004A944F0173016201B1E14B16510461045F
:104FA00071041CF080E1C82ED12CA601B501C4010A
:104FB0000E942A33AC0CBD1C0D2C000CEE08FF081F
:104FC0004C185D086E087F080150104019F7609674
:104FD000E0E10C943A326FEF85E290E00E943933C1
:104FE0006FEF86E290E00E9439336FEF87E290E046
:104FF0000E94393360E088E290E00E9439330E94D9
:105000004B16B0DF6AE885E290E00E9439336FE228
:1050100086E290E00E9439336BE687E290E00C94E0
:1050200039338F929F92AF92BF92CF92DF92EF92DD
:10503000FF920F93CF93DF9388E090E00E9420339C
:105040004B015C01CDE7D4E068839982AA82BB82E0
:105050001C821D821E821F8283E290E00E94183310
:10506000282F30E040E050E060E070E080E090E029
:1050700000E20E945332282939294A295B292883D2
:1050800039834A835B836C837D838E839F83DF9127
:10509000CF910F91FF90EF90DF90CF90BF90AF90A6
:1050A0009F908F900895AAE0B0E0E9E5F8E20C94B3
:1050B0002032FE0131968AE0DF011D928A95E9F7E0
:1050C00006E611E095E7C92E91E0D92EEE24E3948F
:1050D000F12C9E2E8F2EAA24A394B12CF80181913D
:1050E0008F018F3F09F44BC0F894E82FE295EF70E1
:1050F000F0E021A18F70A50102C0440F551F8A95D1
:10510000E2F7CA01922F982B91A392A1809589234F
:1051100082A3789400C0A5E7B1E0692C782C9701B0
:10512000209530956D91F301819191913F016F3FF1
:1051300009F44BC0462F42954F70405E50E0FA0193
:10514000408150E06F7002C0559547956A95E2F72F
:1051500040FD3BC08E299F29A30142505109FA010D
:1051600091838083F1E0AA37BF07E1F6F8018291CD
:105170008F3F11F00E94C00740EA4A95F1F7EE0C0C
:10518000FF1CC016D10609F0A9CF4AE050E0692DF6
:10519000782D83E493E00E94F432892BC9F08AE0F1
:1051A000E92DF82DA3E4B3E001900D928A95E1F783
:1051B00081E0809312020E94AD0C909311028093C3
:1051C00010022A96EEE00C943C3282239323C4CF43
:1051D000809112028115A9F3009110021091110221
:1051E0000E94AD0C801B910B059758F34AE050E0EC
:1051F00063E473E086E693E00E94F432892B49F081
:105200008AE0E3E4F3E0A6E6B3E001900D928A952C
:10521000E1F710921202D5CFCDB7DEB7AC970FB63B
:10522000F894DEBF0FBECDBF85B7806885BF85B758
:10523000806885BF84B7877F84BF0FB6F894A89530
:1052400080916000886180936000109260000FBEC2
:1052500080E890E00FB6F89480936100909361002D
:105260000FBE81E0809321018EEB97E09093E701E0
:105270008093E6010E94C7150E940B160E94D20D72
:105280000E942F0E8091E20084608093E200789467
:1052900080917203811599F08091E9001091EC00E2
:1052A0008F70179511271795182B1092E900809190
:1052B000E80083FD0E943C111F701093E90082E01A
:1052C00084BD93E095BD9AEF97BD80936E000E94D8
:1052D0000615811101C07FDE06E611E0D8018D912F
:1052E0008D018F3F11F00E94C007B1E005371B0709
:1052F000A9F705E711E08AE7E82E81E0F82EF8012A
:1053000081918F018F3F11F00E94C007E016F106D6
:10531000B1F78AE0E6E6F3E0DF01282F1D922A9537
:10532000E9F7E3E4F3E0DF011D928A95E9F780E015
:1053300090E00E942533833E9E4F21F40E94061583
:1053400081112FC063EE7EEF80E090E00E94533326
:1053500060E082E090E00E94393381E080933E0576
:1053600061E083E090E00E94393360E074E184E022
:1053700090E00E9453331982CE0101960E946B0F78
:105380000E946B1728DE40E050E0BA018FE090E009
:105390000E944B3340E050E0BA0183E190E00E946C
:1053A0004B3382E090E00E9418338093500384E0F6
:1053B00090E00E942533909341058093400573DE71
:1053C000EFEFF6E721E0E150F0402040E1F700C0C8
:1053D000000069DE8091660380FF08C06FEF7FEFF9
:1053E00080E090E00E9453330E94CE0E83E090E074
:1053F0000E9418330E94F0043F9A4798269A2E98EC
:1054000082E28093800089E1809381008FEF9FEF9B
:1054100090938700809386000E94FF130E94FF13E1
:1054200080914D0381111EC08DE794E0FADD8091DB
:105430007D04843028F40E946B178DE794E0F1DD41
:105440000E946F0810927C040E94540B80917D048E
:1054500080FF05C060E0869586950E94371881E040
:1054600080934D0380914005806880934005609152
:1054700040057091410584E090E00E94533382E141
:1054800091E090939A03809399038091720310E4C2
:10549000853009F490C007DE11E5812E13E0912ECE
:1054A00006E6402E03E0502ED201F4012191319105
:1054B0008D919D9143E0EB35F40709F48AC02817DC
:1054C0003907A1F3B6E6AB2EB3E0BB2E10E0D50151
:1054D000ED90FD905D01F401619071904F016E14AB
:1054E0007F0449F16E247F2400E0CC24C394D12CA6
:1054F000C3018C219D21892BB1F009831A830E945D
:10550000AD0C9C838B83F1E0FD8391E097012C210E
:105510003D21232B09F490E09E8349815A816B81C0
:105520007C818D816BDA0F5FCC0CDD1C0F3001F7B5
:10553000F401F292E2921F5F153049F60E941C0DB1
:105540004DC080917203843049F180E00E94040BC9
:1055500080E00E94EA0410924E0388E190E00FB6CA
:10556000F894A895809360000FBE1093600083B7F5
:10557000817F846083BF83B7816083BF789488957F
:1055800083B78E7F83BF0FB6F894A8958091600093
:10559000886180936000109260000FBE84DDE6E6B3
:1055A000F3E081919191892B09F033C5A0E7B3E035
:1055B000AE17BF07B1F780917203853009F4C1CFF0
:1055C0000E9409110E94FF130E94EB0B0E94EA0443
:1055D00062CF2817390709F075CF3EDC8091220190
:1055E000811511F1E0903C05F0903D05E114F104C6
:1055F000D9F00E94AD0C8E199F092091CF043091F3
:10560000D0042817390780F49091D2048091D104F6
:10561000981709F4ADC045D91092D0041092CF0468
:1056200010923D0510923C0580917504811569F03A
:105630000E94AD0C2091760430917704821B930B6D
:105640008F3F9F4710F40E94001180917C048115C8
:1056500009F444C080917B04E0917D04E695E695D1
:10566000E81BE0935D03853109F4DFC008F095C0C5
:10567000893009F4D0C008F083C0823009F4B9C081
:10568000863009F4BFC0E0EDEE2EE7E0FE2E09ED16
:1056900017E080915E03811561F010925E030E9415
:1056A000AD0C90935C0380935B03109260031092A7
:1056B0005F030E94AD0C20915B0330915C03821B61
:1056C000930B8F3F9F4750F42E0D3F1D30935C038B
:1056D00020935B038BE593E0F80109950E94EB0BA7
:1056E000F82E80916103F81639F0F09261030E9460
:1056F0001C0D8F2D0E94EA0480917203843009F002
:10570000C4CE83E08093E9008091E80082FFBDCEA3
:105710008091E80090E085FF06C00E94A10D8115F0
:1057200009F48CC091E08091E8008B778093E800C9
:10573000911509F4AACEE0907503F0907603E98103
:10574000E114F10409F499C0EE3F09F0B9C08A816F
:10575000833020F08550833008F0B2C0EA81EE300B
:1057600008F0AEC0F0E0E55FFB4CCE0101963BC611
:1057700052D810923D0510923C050E94610B54CF07
:105780008F3009F080CFE695F0E0E75DF94FE491C6
:10579000EE2EF12C02E219E07CCF74EFE72EFF240D
:1057A000F39404E41AE0843209F473CF90F468E2CD
:1057B000E62EF12C04EC19E0883109F46ACF83322B
:1057C00009F061CFE4E2F6E0E590F5900FEA18E029
:1057D00060CF853209F057CF8E2F63E0C4D5E92F13
:1057E000F0E0EF5DF94FE491EE2EF12C09EB16E1BC
:1057F00050CFF0E0EE5CF94FE491EE2EF12C09EE83
:1058000018E047CFF0E0E15DF94FE491EE2EF12C86
:105810000AED18E03ECFE695F0E0E45DF94FE49143
:10582000EE2EF12C0CEF18E034CFF0E0EA5DF94FEA
:10583000E491EE2EF12C0CE719E02BCF50E2C52EAF
:10584000D12C9E012F5F3F4F79018091E80085FDAB
:105850000AC08091E8008B778093E8000E94A10D38
:10586000811599F35FCF8091F100D7018D937D0170
:10587000B1E0CB1AD10849F755CFE43148F4E1152E
:1058800051F0E150E33138F4F0E0E75EFB4CABC59A
:10589000EE3F09F463CF8FEF898312C01A8289E04B
:1058A0008B830EC08A81823081F08330B1F08130E9
:1058B00091F70E941C0DADD56B837C838D839E83F5
:1058C000CE0101960E94F10DE0CD88E290E0B0D6C5
:1058D0001B821C821D828E83F3CF80917003909176
:1058E0007103892B69F3FE013196D2018C911196D7
:1058F0009C91B2E04B0E511C92838383329620E739
:10590000421623E0520689F7DBCF8A81823019F6EE
:105910006B817C818D819E817CD588E290E0A9D6C7
:10592000CFCF4C816B818A810E94211498278927CF
:1059300098279E838D83C4CF2D813E8132272327D4
:1059400032274C816B818A810E94710FB9CF0E94EE
:105950004B16B6CF8A81893059F48B8136E0839F0C
:10596000C00111246FEF70E017D5862F0E94040B41
:105970008A81823891F1B0F48038E9F0813809F0F9
:105980009FCF60E08B810E9437189B8180917D04BE
:1059900091111AC08E7F80937D0410927C040E9426
:1059A0007D088ECF833809F08BCF20E040918004B2
:1059B0006C818B8106C020E04B8160917F048091D7
:1059C0007E040E948A177CCF816080937D0460E012
:1059D000869586950E94371873CF8B8180938104BA
:1059E0006FCF8A81893089F08A30E9F0823861F19D
:1059F000E0F4803821F1813809F062CF80917D0494
:105A000080FF20C0869586954BCF80917404869543
:105A1000869586954FEF849FC001112466E070E063
:105A2000BBD46B834DCF1B824BCF833809F048CF5B
:105A300080917E048B8380917F048C8341CF809101
:105A400080042ECF80E02CCF8091810429CF84E781
:105A500094E00E946B0F0E946F088DE794E00E9413
:105A60004A172ECF80E18A832BCF1A828FEF18CF6F
:105A70008C818D3108F024CF8A809B8098248924E2
:105A80009824A12CB12C8E010F5F1F4F7801E80ED6
:105A9000F11CE016F10609F413CF8FEF881691047C
:105AA000A104B10478F4C4018F5F9C4FC1D5D80123
:105AB00014968C930F5F1F4FBFEF8B1A9B0AAB0A94
:105AC000BB0AE7CF80E0F3CF809170039091710320
:105AD000892B09F4F5CE8C818D3108F0F1CE882E1A
:105AE000912CA12CB12CCA80DB80DC24CD24DC24B9
:105AF000E12CF12C8E010F5F1F4F412C512C3201F4
:105B0000481459046A047B0408F0DACEEFEFCE168D
:105B1000D104E104F10438F4D80114966C91C60163
:105B20008F5F9C4FA6D5BFEF4B1A5B0A6B0A7B0AAF
:105B3000EFEFCE1ADE0AEE0AFE0A0F5F1F4FE0CF2C
:105B400011DABECE84E08FCF8C818D3108F0B8CED3
:105B5000882E912CA12CB12CCA80DB80DC24CD2492
:105B6000DC24E12CF12C412C512C32018E010B5FF5
:105B70001F4F481459046A047B0408F0A1CE80E04A
:105B8000F8E5CF16F2E0DF06E104F10418F4C601EF
:105B900089964ED5D8018D938D01BFEF4B1A5B0AC4
:105BA0006B0A7B0AEFEFCE1ADE0AEE0AFE0AE1CF9D
:105BB0002C81022F10E02D3108F082CE8A819B814A
:105BC0009827892798272C01612C712C8835F2E0C1
:105BD0009F0708F075CE822E912CA12CB12C48E5A0
:105BE00052E060E070E044195509660977094217F0
:105BF00051056105710508F463CE20917003309161
:105C00007103232B09F03EC01C0129E2220E311C36
:105C100080FBEE24FF24E0F880FF0BC0889608D5B7
:105C20009D8189279827892781159C4711F48FEF3B
:105C30008D83D501C401840D951DA61DB71D80FF60
:105C400019C0680141E0C41AD108CE0105968C0D37
:105C50009D1D9CA78BA7C101800F911FE9D4ABA507
:105C6000BCA59C9181159C4721F48FEFEBA5FCA569
:105C700080838601FE013196EE0DFF1D2FEFE016A9
:105C8000F10638F08E010F5F1F4FC12CD12C760129
:105C900025C09481858181159C4711F42483258337
:105CA00042E0E40EF11C3296EACF88E5481682E025
:105CB00058066104710430F4D80114966C91C20145
:105CC0008996D7D4BFEFCB1ADB0AEB0AFB0AEFEFBA
:105CD0004E1A5E0A6E0A7E0A0F5F1F4FC814D9045F
:105CE000EA04FB0410F3ECCD8091700390917103F2
:105CF000892B09F4E5CDCE0101960E94F10DFFEF4D
:105D000021EE34E0F15020403040E1F700C00000C7
:105D10006BCB88E0E3E2F1E0DE01919601900D9219
:105D20008A95E1F7FE0132968FE1DF011D928A9597
:105D3000E9F786E0898388E07F96DE011596019079
:105D40000D928A95E1F7BCCD80E8898382E08A8351
:105D50001B821C82B5CD0B811C81012E000C220BF5
:105D6000330B45E0000F111F221F331F4A95D1F757
:105D7000B901A801405E5F4F6F4F7F4F4017510739
:105D80006207730708F49CCD0038B2E01B072105B9
:105D9000310508F095CD4138E2E05E0761057105F7
:105DA00020F040E852E060E070E0401B510BB80189
:105DB0006A5C794F03D484CD4AE150E06FEF70E024
:105DC000CE0107961ED4809170038983EA821B82DC
:105DD0001C8282E08D838DE07ECD81E090E0909307
:105DE00076038093750382E390E09093650380933C
:105DF00064030E94AD0C909363038093620360CDB3
:105E0000E114F10481F1D0906603C0906B0300911E
:105E10006203109163030E94AD0C801B910B8536C9
:105E2000910540F1C5FE26C0D0FE24C00E94AD0CF5
:105E30009093630380936203809164039091650360
:105E400001979093650380936403892B61F410920A
:105E500076031092750381E090E090937103809334
:105E60007003E12CF12C809170038983EA82809188
:105E7000640316CD82E390E09093650380936403FE
:105E8000F2CF10927103109270031ACD40E250E0ED
:105E90006FEF70E0B6D314CD2B81243009F473C0BA
:105EA00010F5211509F462C0233009F009CD2C81C9
:105EB0006AE0CE018196FC01362F11923A95E9F7FE
:105EC000283008F05EC0629FB00111246F577D4FEB
:105ED0004AE050E09DD380E089838AE0FE01B196DC
:105EE000DE0112962CCF273009F47AC0283009F051
:105EF000E7CC6C8186E0FE013596DE01919601903B
:105F00000D928A95E1F789A19AA18115FCE79F0777
:105F100041F42091700330917103232B11F480E040
:105F200090E09AA389A38BA19CA181152CE79207ED
:105F300041F42091700330917103232B11F480E020
:105F400090E09CA38BA38FEF683060F436E0639FF2
:105F5000B00111246F527D4F46E050E0CE01819692
:105F6000A6D380E089830E940B16AACC2FE1DC0126
:105F70001D922A95E9F788E08A838C8383E088A3C1
:105F80009FCC8FEFA9CF6C818AE0FE013596DE01B0
:105F9000919601900D928A95E1F789A59AA58115B0
:105FA0004CE7940741F42091700330917103232B47
:105FB00011F480E090E09AA789A78FEF683060F431
:105FC0008AE0689FB00111246F577D4F4AE050E08E
:105FD000CE0181966CD380E089830E94C71570CC76
:105FE0002C8166E0CE018196DC01E62F1D92EA95B8
:105FF000E9F7283060F4629FB00111246F527D4FA1
:1060000046E050E005D380E0898386E067CF8FEFDC
:10601000FBCF80914F03811509F4CDCAB0E1B9BD22
:10602000E2E1E9BD09B400FEFDCF8091D8008F7D8B
:106030008093D8008091E00082608093E00080919E
:10604000E00081FDFCCF0E940911B5CA1F921FB666
:106050001F9211248F939F93AF93BF9380914E0310
:10606000811113C08091280290912902A0912A02E7
:10607000B0912B024196A11DB11D809328029093EF
:106080002902A0932A02B0932B02BF91AF919F9156
:106090008F911F901FBE1F90189578941F921FB666
:1060A0001F9211248F939F93AF93BF9380912802E7
:1060B00090912902A0912A02B0912B020196A11D74
:1060C000B11D8093280290932902A0932A02B093D5
:1060D0002B02BF91AF919F918F911F901FBE1F9078
:1060E00018951F920F920FB60F9211242F933F9382
:1060F0004F935F936F937F938F939F93AF93BF93D0
:10610000EF93FF938091E10082FF09C08091E2004C
:1061100082FF05C08091E1008B7F8093E100809138
:10612000DA0080FF24C08091D80080FF20C08091D9
:10613000DA008E7F8093DA008091D90080FFA9C0B9
:1061400080E189BD82E189BD09B400FEFDCF81E017
:106150008093720380911702811109C00E94D20DB1
:106160000E942F0E8091E20084608093E200809173
:10617000E10080FF1AC08091E20080FF16C080918C
:10618000E2008E7F8093E2008091E2008061809344
:10619000E2008091D80080628093D80019BC85E02D
:1061A0008093720383E0809321018091E10084FF5A
:1061B0002FC08091E20084FF2BC080E189BD82E185
:1061C00089BD09B400FEFDCF8091D8008F7D8093FA
:1061D000D8008091E1008F7E8093E1008091E20001
:1061E0008F7E8093E2008091E20081608093E200E4
:1061F00080911602811509F452C084E080937203E5
:1062000080917203843009F052C082E080932101B2
:106210008091E10083FF2CC08091E20083FF28C0C1
:106220008091E100877F8093E10082E08093720398
:10623000109216028091E1008E7F8093E1008091A0
:10624000E2008E7F8093E2008091E2008061809383
:10625000E20042E060E080E00E94FF0D8091F000EB
:1062600088608093F00081E0809321018093200179
:10627000FF91EF91BF91AF919F918F917F916F911E
:106280005F914F913F912F910F900FBE0F901F90F4
:10629000189519BC109272031092170268CF809162
:1062A000E30087FF02C083E0A9CF81E0A7CF81E0B0
:1062B000ADCF1F920F920FB60F921124EF92FF9263
:1062C0000F931F932F933F934F935F936F937F93FE
:1062D0008F939F93AF93BF93CF93EF93FF9309EE69
:1062E00010E0F8018081C091EC008F70C795CC2739
:1062F000C795C82B108280EFE82EF12CF701808122
:10630000877F808378940E943C11F8011082F70106
:10631000808188608083CF70F801C083FF91EF9106
:10632000CF91BF91AF919F918F917F916F915F912D
:106330004F913F912F911F910F91FF90EF900F90F0
:106340000FBE0F901F901895DB018F939F93E2D1A2
:10635000BF91AF91A29F800D911DA39F900DB29F01
:10636000900D11240895992778E0880F991F9617AA
:1063700008F0961B881F7A95C9F78095089587FBCA
:10638000082E062687FD819567FD6195ECDF0EF4EA
:10639000919507FC81950895AA1BBB1B51E107C08D
:1063A000AA1FBB1FA617B70710F0A61BB70B881FA5
:1063B000991F5A95A9F780959095BC01CD01089534
:1063C00097FB072E16F4009406D077FD08D0E4DF83
:1063D00007FC05D03EF4909581959F4F08957095E8
:1063E00061957F4F0895EE0FFF1F0590F491E02D0A
:1063F0000994082E817006940694811D0694811DCF
:106400000694811D0694811D0694811D0694801DAD
:106410000895692796276927782787277827089579
:10642000ABD1332312F48A1B9B0B01C0A5D1B7FF5C
:106430000895821B930B08952F923F924F925F9283
:106440006F927F928F929F92AF92BF92CF92DF9284
:10645000EF92FF920F931F93CF93DF93CDB7DEB7E9
:10646000CA1BDB0B0FB6F894DEBF0FBECDBF09947D
:106470002A88398848885F846E847D848C849B84D4
:10648000AA84B984C884DF80EE80FD800C811B81E2
:10649000AA81B981CE0FD11D0FB6F894DEBF0FBE11
:1064A000CDBFED010895002E083090F0982F872F72
:1064B000762F652F542F432F322F22270850F4CFE9
:1064C000220F331F441F551F661F771F881F991FF8
:1064D0000A95B2F7002D089597FD1094002E08300C
:1064E00098F00850232F342F452F562F672F782FE1
:1064F000892F912DF4CF159497958795779567956A
:1065000057954795379527950A95AAF71124002D99
:1065100008958F929F92AF92BF92CF92DF92EF92A7
:10652000FF92CF93DF93EC01688179818A819B810F
:10653000611571058105910521F464E279ED8BE522
:1065400097E02DE133EF41E050E0C8D049015A0116
:106550009B01AC01A7EAB1E4DDD06B017C01ACEE9C
:10656000B4EFA5019401E2D0DC01CB018C0D9D1D9F
:10657000AE1DBF1DB7FF03C00197A109B0488883B6
:106580009983AA83BB839F77DF91CF91FF90EF9090
:10659000DF90CF90BF90AF909F908F900895B9CF2C
:1065A00080E091E0B6CFA0E0B0E08093000190934E
:1065B0000101A0930201B09303010895FB01DC01E6
:1065C00002C005900D9241505040D8F70895FC014B
:1065D0004150504030F001900616D1F73197CF016D
:1065E0000895882799270895FB01DC0104C08D9147
:1065F0000190801921F441505040C8F7881B990B35
:106600000895DC0101C06D9341505040E0F70895BA
:10661000DC01CB01FC01F999FECF06C0F2BDE1BD62
:10662000F89A319600B40D9241505040B8F7089551
:10663000F999FECF92BD81BDF89A992780B508954A
:10664000A6E1B0E044E050E0E5CFA8E1B0E042E0F0
:1066500050E0E0CFDC01A40FB51F4150504040F0A6
:10666000CB01840F951F2E9105D041505040D8F793
:106670000895262FF999FECF92BD81BDF89A019712
:1066800000B4021639F01FBA20BD0FB6F894FA9A7A
:10669000F99A0FBE08950396272FECDFEADF252F26
:1066A000E9DF242FE7CF0196272FE4DFE2CFDC01DB
:1066B000CB0102C02D9105D041505040D8F708952C
:1066C000262FF999FECF1FBA92BD81BD20BD0FB60E
:1066D000F894FA9AF99A0FBE01960895052E97FB41
:1066E00016F400940FD057FD05D024D007FC02D03B
:1066F00046F408C050954095309521953F4F4F4F37
:106700005F4F089590958095709561957F4F8F4F5D
:106710009F4F089531D0A59F900DB49F900DA49FD9
:10672000800D911D11240895B7FFF4CFF3DF821B74
:10673000930B0895A1E21A2EAA1BBB1BFD010DC0ED
:10674000AA1FBB1FEE1FFF1FA217B307E407F50721
:1067500020F0A21BB30BE40BF50B661F771F881FFD
:10676000991F1A9469F760957095809590959B0193
:10677000AC01BD01CF010895A29FB001B39FC0013C
:10678000A39F700D811D1124911DB29F700D811D5D
:106790001124911D0895F894FFCF19123F1245124C
:1067A0003F1245129712B8124512BE13CB13691D42
:1067B000D11D711D3B1D3F1D751D431D791D851D7F
:1067C0004F1DCA1D531D891D571D8D1DB21D5B1DFB
:1067D000911DB91D611D971D9F1D471D7D1D4B1DE1
:1067E000811D651D9B1DA91DC21DC81D351D6D1D6B
:1067F000D81D121D161D081D0E1D1A1D1E1D221D41
:10680000F91D101E141E181E1C1E201E241E281EDC
:106810002C1E301E341E892EA42EAB2E602C602C14
:10682000DC2EED2E002F412F462F602C602C602C8B
:106830004C2F4E2C522C852C912C9C2CA72CAA2C06
:10684000F12C272D4B2C742E322D352D382D642D07
:08685000A02DA22DA42DD82DCE
:106858000100000001010201191A1B1C1D1E1F2046
:106868002122AA0C340F4A0F280D4F0F2B0F0000BE
:10687800010001176441C15FCA48DD0044226D3B35
:10688800011901AC0041025A027A02000102020217
:10689800020606060909090909090F0F0F0F0F0F4C
:1068A8001515151819191919191919191919232448
:1068B800252525252525909192939594969734F72B
:1068C800F6F5F4F1F03031323337E200E900EA004E
:1068D800B500B600B700CD008301CC008A01920153
:1068E80094012102230224022502260227022A02F9
:1068F800B300B4006F0070009F01CB019F02A0029B
:10690800E200E900EA00B500B600B700CD00830157
:10691800CC008A019201940121022302240225025B
:10692800260227022A02B300B4006F0070009F01FC
:06693800CB019F02A0024A
:00000001FF
